:10720300DFAE9F9EDF8E9F865E867F867F867F8E24
:107213009F969EA6DFA6DFAEFFAEFFB71FBF3FC799
:107223003FC73FC73FCF1FC73FBF3FB73FBF1FBE8C
:10723300FFAF1EAF1EAEFEAEFEA6DEA6BEAEBEA660
:10724300DFAEDFAE9DC6DDE79FCF1EA69E969F8E67
:107253007F8E9F867F7E5F7E5F765F6E1F661E5E7C
:107263003E663E663F665F665F5E3F561E4E1F4E3E
:107273001F4E1F4E1F4E1F4E1F4E1F4DFF4DFE56DE
:107283003F5E5F5E5E667E665E661D55FD4DDE4D4E
:10729300DE4DDE4DFF4DFF4DFF4DFF4DFF4DFF4DCD
:1072A300FF4DFF4DFF4DFE4DFE4DFF4DFF4DFE4D7E
:1072B300FE4DFE55FE55FE55FE4DFF4DFF4DFF4D58
:1072C300FF4DDF4DDF4DDF4DDF4DDF4DDF4DDF4D3B
:1072D300DF4DDF4DDF4DDF4DDF4DDF4DDF4DDF4D4B
:1072E300DF4DDF4DDF4DDFBEBCBEFDAEFD9F1E8E0D
:1072F300DE96BD9EBEA6BEA6BEAEDEAEDEB6FEB6B4
:10730300FEAF1EA6DE9E9DA6BEAEBDAEBDA6BDA6AD
:10731300BDAE9DAE9DC77FD79FDFBFDFBFDFBFE79A
:107323009FE7BFD75DB6BC9E9D8E5D7E3D7E1C7D77
:10733300FBB73EDFDFDF9FDF9EDFBFD7DF869D65C5
:10734300FC763E761F6DBD96BECFFFD7BEDFBECFA8
:10735300DF867C4DBC4DDF559D96DED7FFDF9EDF7C
:10736300BF967E559D4DDD5DDBB77EDF9EDF9FB60D
:107373009CAE7BD75EF7FFFFFFF7DEE79EDF7EC69F
:10738300DBD77ED7BFAE9DA63DA65EA65DAE5DB63E
:107393009EB6BEBF1FC75FAEDE8E5E965E967F96BD
:1073A3009F967E967E8E3E865E7E5E765E661D6EC2
:1073B3001D6E5E765F763E763E867E96BE969E9E7A
:1073C3009E9E9E9EBEA6BFA6BFA6BFA69EA69EA627
:1073D3009E9E5DA67DA67EA69EA69F9E9E9E9F9632
:1073E3009F969F967E8E7E8E7E967E967E969E9EA0
:1073F300BE9EBFA6BFA6DF9EDF9EDF96FF9EFE9EBC
:10740300DE9EDE9EBF9E9E9E9E96BF8E9F969F9EF5
:107413005E865F867F8E5E965E9E7F9E9F9E9F9614
:107423009F969EAEBECF5FCF7FA6BE7E5E6E3E5E54
:107433001E561E561E561E4E1E4E1F4E1F461F4ED6
:107443001F4E1F4E1F4E1F4E1F461F463F4E3F4EA1
:107453001F4E1F4E1F4E1F4E1F561F4E1F463F46A9
:107463003F4E3F4E1F4DFF4DFF4E1F4E1F4E1F4EB3
:107473001F4E1F4E1F4E1F4E1F4E1F461F4E1F4DAA
:10748300FF4DFF4DFF45FF45FF45FF4DFF4E1F5687
:107493003F5E3F5E5F665F5E3F561F4E1F4DFF4D73
:1074A300FF4DFF4DFF4DFF4DFF4DFF4DFF4DFF4D79
:1074B300FF4DFF4DFF4DFF4DFF4DFF4DFF4DFF4D69
:1074C300FF4DFF4DFF4DFF43B44CB95D7D6DBBCF09
:1074D3007FF7FFFFFFFFFFFFFEFFFFFFFFFFDFF76A
:1074E300DFE7FF8E7D559C5E1E65FE761E7E3E7E2B
:1074F3005F863E963DDFBFEFFFF7FEFFDEFFBFF780
:10750300BFF7DFEF9FCEFEBEDFAEBFB6BFBF1FAE7E
:10751300FFBEFEEFDFF7BEF7BEEFBEEFFFAF7F5557
:107523009C55DE4DFF4DDE65DCBF5EE7DEEF9DDF84
:10753300BEBF9F6E1D55FE5DFD6E1BB77FCF9FCFF8
:10754300BEBFBF8E9D7E3D965CC6FDEFDFEFDFF7CE
:10755300FFFFFEFFBEFFBEF7DFF7FFFFDEFFFFEF1C
:107563009EE77ED77ECF5FBF1FBF1FBEFFBEFFA6B6
:107573007EA67EAEBFA69E9E5DA69EA6BEAEDEA6E0
:10758300BE9E7D9E7E9E7E9EBE9EBE9EFE9EDE9681
:10759300BD9EDE9EDE9EBE969E9EBEAEDFB6DEB670
:1075A300FFB6FFB6FFAEDFAEDFAEFFAEFFAEFFAEA0
:1075B300FFAEDFAEDFA6DFA6BF9EBF9EBF96BF9620
:1075C3009F969F967F9E9FA6BFA6BE9EBE9EBE9E73
:1075D300BE969E869E763E661D5E1D5E1E5E1D5E8B
:1075E3001D5E1D5E1D6E5D663D563D563E5E1E6D07
:1075F300FD761D75FC8E5DA6FF96DF869F6E7F660A
:107603003E867E9EFF9E9F7E1D5DFD561E4E1E4E38
:107613001E4E3E4E3F4E3F4E3F4E3F4E3F463F4E29
:107623003F4E3F4E3F4E3F4E3F4E3F4E3F4E3F56E7
:107633001F4E3F4E3F4E3F4E3F4E3F4E3F4E3F4607
:107643003F4E1F461F461F4E1F4E1F4E1F4E1F4EBF
:107653001F4E1F4E1F4E1F4E1F4E1F4DFE4E1F56D9
:107663001F55FE5DFE5DFE55FE4DFE4E1F4DFE4D4C
:10767300FE561F4DFF4DFE55FF4DFF4DFF4DFF4D78
:10768300FF4DFF4DFF4DFF4DFF4DFF4DFF4DFF4D97
:10769300FF4DFF4DFF4DFF4DFF4DFF4DFF4E1F4E65
:1076A3001F4E1F4E1F4DFF95BA54155C779E3DDF4D
:1076B3007FF7DFF7DEF7DEF7DEF7BEF7DFF7DFF79B
:1076C300BEF7DFAEBD5DDD561F561F5DFF6E1F6E3D
:1076D3003F661F7DFDB71EE7FFEFDEF7DEF7BFF75F
:1076E300BEEFDFEFDFBEBDA65DA67DA69DAEBDAE40
:1076F3003CAE3BD79FD7DFCFBFCFBFD7BFB75F8EE0
:107703009D8EBD86DE86DE8E9DAEFEB71FAF1FA6A5
:10771300DEA69DB75EBF5EBF5EC77E9EBD7E1C8636
:107723005C9E9CC73EE79FEFBFF7BEFFBDF7DFEF51
:10773300BFF7BFFFDFFFDFFFDFFFDFFFDEF7DEFFA8
:10774300FFEFFFD73EBEFEBF3EB71FB6FEAEBEA6DF
:107753007DAEDEAEBE9E5DA67DAE7CBEFDD77FCF89
:107763007EC71DC71EC73FCF3FCF1EC6FEC71FC75D
:107773003FC71FC71FC73FC73FC71FC73FCF3FC72E
:107783001FC71FC71FBF1FB6FFB6FFB6FFAEFFAEB3
:10779300DFAEDFA69EA69EA69EAEBEAEDFAEDFA682
:1077A300BEA6BEAEBFAEDFAEFFAEFEA6FFA6FF9681
:1077B300BF7E5E6E5F665E563F4E3F4E3F563F5600
:1077C3003F65FCA6FDBFBF869C65DA863CAEFEC75F
:1077D3005FD77FCF3ED77FC77F9E9E7E1D6E3E5D68
:1077E300FD6DFD7E3E75FE661E563F4E3F463F4E87
:1077F3001F4E1F4E1F4E1F4E1F4E1F4E1F4E1F4E1E
:107803001F4E3F4E3F4E1F4E1F4E1F4E3F4E3F4E8D
:107813003F4E3F4E1E4E1E463E3E3E465E563E5E2B
:107823003E665E6E5E6E5E665E5E3E4E3E4E3E4EF5
:107833003E4E1E4E1E4E1E4E1E4E1E4E1E5E3F667C
:107843007F6E9F767F6E7F663E561E4E1F4E1F4D88
:10785300FF4DFF4DFF4DFF4DFF4DFF4DFF4DFF4DC5
:10786300FF4DFF4DFF4DFF4DFF4DFF4DFF4DFF4DB5
:10787300FF4DFF4DFF4DFF4DFF4DFF4DDE55DE55D7
:10788300DE55BE4DDF4DFF9578955784B49D16E7C1
:107893005EFFFFF7DFFFDFFFFFFFFFFFFFFFFFF7E6
:1078A300DFF7FFCF3E965D763D661D6E1D761D7636
:1078B3003D7E5E861CA6DDD79FDF5FE77FE77EEF19
:1078C3007FEF9FEF9FE7BFDF7ED75ECF3ECF5EC7E1
:1078D3003DC75EA6DD7E1C661D663D6E1C6DDBA787
:1078E3001DE7FFF7DEF7BEEFFFC79F7E1D763E86DF
:1078F3007F8E5DCF7FEFFFEFBFEFDFCF9F9E9D9E1C
:107903007E9E9EB6DDDFBFF7BFFFBFFFDEFFDFFF5B
:10791300DFFFDFFFDFFFDFFFFFFFDFFFBEF7BDEFAF
:10792300BEE79ECEDDDF5EDF9EB6DDB6DDD75ED77A
:107933003DE7BFDF9FCF5ED77ED75EEFFFF7FFFF49
:10794300FFFFFFF7DEF7FFF7DFEFBFDF5EDF7ECF7F
:107953001EBEFEB6DDB6DEB6FEBF1FBF1FBF1FBE17
:10796300FEBEFEBEDEBEFFB71FB6FFB6FFB6FFBF4D
:107973001FB6FFB6DEB6DDB6DEBF1EC73FC73FC7C5
:107983003FC71EBEFEBEDEB6DEB6FFAEFF969E7ED0
:107993005E767E765E6E5E6E7E6E5E6E5E6E5D6E35
:1079A3005D7DFACF3ECF5F8E5B8E9BCF7FF7DFEFA0
:1079B300DFEF9FE77FD75FB6BD9E7D9EBF867E8646
:1079C3003D967E9EBF9EDF96DF869E765E6E7F6EC1
:1079D3007F667E667F665E5E5E5E7E5E7E5E7E5EEA
:1079E3005E5E5E5E7E567F567F565F565E563E5E99
:1079F3005E6E3D869E8EBE869E7E9F76BF767E7E23
:107A03009E867E8E7E867E767E665D565D563E5E65
:107A13003E5E3E5E3F563E563E565E563E5E3E5E82
:107A23003E5E5E5E5E563E5E3E565E4E5E563E5623
:107A33003E561E563E563E4E3E563E563E563E56CB
:107A43003F4E1E4E1F4E1F561F561E561E563E4E6F
:107A53003F563F563F561F5DFD763D96DEA6FEA67A
:107A6300FF96BF7E7E663FBE5ABE5ACE9BADB89D83
:107A730015BE3AE7BFDF5ED73ECF3EC6FEBEDEB6DB
:107A8300BDBE9DCF1EDF9FD79ECF7ED79ED79EDFE5
:107A9300BFE7BFE7DFDF7EBE5CBE5DBE9EC6DFCE57
:107AA300DED6FEC69DD6FDF7DFF7DFFFDFFFFEFF65
:107AB300FFF7FFCF7F861C763E661F65FE7DDCAE3B
:107AC300BCE7DFEF9EF7BFEFDFDFFFA6DE7E1D869D
:107AD3003E965DAEBCDF9FDF9ED77ECF7EBF5EC787
:107AE3005ECF3ED75EEFBFFFDFFFBFFFDFFFDFFFEE
:107AF300DFFFDFFFDEF7DFF79FEF9FF7FFF7FFEF14
:107B0300DFD6FDCEDDE79FEFDFE79EEF9FF7DFFFD9
:107B1300FFFFFFF7DFF7DFEFDFEFDFEFBFF7DFFF9A
:107B2300DEFFDEFFFFFFDFFFDFF7BFF7BFF7BFE7D4
:107B33009FE7BFD75EC6FDB6DDB6FDBF1EBF3EBF26
:107B43003EBF1EBF1EBF1EBEFEBEFEBEFEBEFEC7A6
:107B53001EC71EC73ECF5FCF7FCF5FCF3ECF3EC78F
:107B63001EC71EC71EBF1EBF1EBF1EAEFDA6DD9EC7
:107B7300BC9EDD9EFDA6FDA6FD9E9CAEFDBF5ECF19
:107B83005ED77EDF5EDF7ECF9FAEDCC6FDE77FDFA5
:107B93005ECF3ED77EBEFDB6FDBF1EBF3EB6FEB670
:107BA300FEB71EAEFEAEFDA6BCA6BCA6DD9EDD9650
:107BB300BC96BC96DD96BD8EBC8EBC8EBD8EBD8E36
:107BC300BC86BD86BC86BC86BC8EBC8EBC96BCA661
:107BD300DDAF3EB75EB71DB6FDAE9CAE9C9EBC9EB0
:107BE300BC9EBC8E5B965CAEFDB71EAEFEA6FE963B
:107BF300DD7E9C7EBD76BD7E9D7E9D769D769D764B
:107C03009D769D769D769D769D769D7E9D86DD8671
:107C1300BD86BE7EBE769D6E9D6E9D6E9D6E9D6E77
:107C23007D6E7D6E7D6E7D6E7D667D667D667D6619
:107C33007D667D6E5C769DA71EBF3FB6FEBF3FB7D8
:107C43003F9EFE86DE769E8D168D168CF68D1695DE
:107C530038324D5BD39DDB95FC8DDC85DD7DFE8667
:107C63001E85FD9E3DE7BFFFFFFFDEFFDEFFFFFF3B
:107C7300DEFFDDFFDEEFBFB65DA63EA67F9E5FA6FD
:107C83005EAE7EAE5DB65BE79EF7DFF7DEFFDEFF3F
:107C9300DEF7DFDFBFAE9DA69DA6BFAEFFCF5FDFE2
:107CA3009FE7BFEFBFEFBFEFDFE7BEDFBFD77FCFFA
:107CB3005FDF9FE7BFE79ECF1DBEFDAE7CBEDCE767
:107CC300DFF7FFFFDFFFDEF7BFF7BFFF9FFFBFFF5A
:107CD300DFF7DEF7FFE77ED6BDD6DDDF5FDF9FD7B9
:107CE3007ED75EDF5DEF9FEF7EF7BFFFDFF7BEFF5F
:107CF300BEFFDFF7BFEFBFE77FEF7FEF9FF7BEFF6B
:107D0300BEFFBEFFBFF7BFF7BFF79FEF9FE75EDF83
:107D13003EE79FEFBFDF9FC73FC73FC73FC73FBF99
:107D23001EC71FBF1FBF1FB6FFB6DEB6DEB6DEB669
:107D3300DEB6DEB6DEAEDFB6FFB6DEAEBEAEBEB6D6
:107D4300BEB6DFB6FFAEDFB6DFAEBEAE9DAEBDB62E
:107D5300BDC73EE7BFE79FCF1DCEFCDF5EEFBFF79A
:107D6300DFFFDFF79EE77EE7BFC6DDBE9DC6FEC62B
:107D7300BDB6BEAEBE9E7D967D967D965D967E8E8D
:107D83005E8E3E8E1D8E3D9E7D9E7DA69DA69D96FE
:107D93007D969D8E5D7E1C7E3D8EBE869E7E3E764E
:107DA3001E763E763D763D7E5E865E969EAEBFAE89
:107DB300BF9EDF8E9E7E5C75FB7E3CA6BEBEBEBEB6
:107DC300DFAEFF9EBE9EBEAF1EB6DEA6BE8E9E7605
:107DD3005D563D4E5D4E3D4E1E55FE4E1E4E1E4E95
:107DE3001E4E3E4E3E4E1D4E3E5E1D6E3D767E7ECB
:107DF3007E765E663E5E1D561D561D561D561E56EC
:107E03001E561E55FE5E1E5DFF5DFE5E1E5E1E66F9
:107E13001E6E1E6DFE7E3E867E863E7DFD75DC6D8E
:107E2300DC5DBC55DD661E63F4641474766C559595
:107E33007A4331222D2AB0649785FE7E1E75DE7546
:107E4300FE75DE963DD79FF7DEFFDEFFDFF7DFF738
:107E5300DEF7DEF7FFE7FFBEDEA67EA6BF9E7EAEA1
:107E63007EB6BEB6BEBEBDD75EDF9EDF9FDF7FD7C9
:107E73005ECF3FC71ED73EE79EF7BEF7BFF7DFEFE4
:107E8300DFE77ED71EDF3FE75EE75DE75DFFBEFF0F
:107E9300FFFFFFFFFFF7DFE7BFC71EBEDED73EEFE3
:107EA300BFFFFFFFDFFFDFFFDFF7DFF7BFF7BFF73F
:107EB300DFEFBFE79FD71EDF7FE79FDF5EBE9DAE8D
:107EC3005DBEBDE7DFF7DFF7BFF79FF7BFEFBFEF9C
:107ED3009FE77FDF5FD73FCEFEDF3FEF7FF7BFF741
:107EE300BEEF9EEF9FE77FDF7FD73FC6FEC6BEC6CE
:107EF300FFC71FC73FBEFEB6DFBEFFBF1FBEFFB635
:107F0300FFB6FFB6FFAEFFA6FFA6DFA6DFA6DFA67E
:107F1300DFA6DFA6DF9EBF9EBF9EBF9E9FA6BFA616
:107F2300DFA6BFA69EA69EAEBFA69EAE9EBEDED712
:107F33007FE7BFEF7FEF5FEF7FEF9FE77FE75EE7CF
:107F43007EEF7EEF7EDF7EDF5FDF5FC75FBF3FAE2B
:107F53009EA69F969F969F8EBF869E7E7E869F86B9
:107F63007EA6BEB73FC75FCF9FCF5FCF3FCF5FD761
:107F73007FCF5FCF5FBEFEBF1FB73FAEDF9EDF8EFB
:107F8300DF8EBF86BF86BF869E867E8E9F867E8659
:107F93007E869E7E9E867E967EAEFFB6FFC6DFB64B
:107FA300BFA69EA6FF96FE8E9D8E7C8E5D8E5E7E08
:107FB3007E767E6E9F6E9F6E7F6E5F6E5E6E7E665A
:107FC3005E663E665E665E6E7F6E7E6E5D6E3D6E67
:107FD3003D6E5E6E5E6E7E667E6E7F6E5E6E5E6E06
:107FE3005F6E5F6E3F6E5F6E5F765F767F769F76C6
:107FF3009F767F7E7F7E7F7E7F7E9F7E9F7E9F7E1E
:108003007E7E7F867F8EBF84D784B663927C55AD98
:10801300DB4B303ACF2A8E1A4D3B52757B865E8EF0
:108023005E965FAE9DD79FF7FFF7DFF7DFF7DFEFD2
:10803300DFDF9FDF9ECF5EBEDDBEDDC6FDD73EDF49
:108043007EE79FE79EE7BFCEFDAE3CB69EAE7E9E2B
:108053005D9E9F8E1DBEFEF7FFFFBEFFBEFFDEFFD0
:10806300FFE79FC6BEC6DED73EEF7FEF9FF7BEF7A3
:10807300FFF7DFFFDEFFBEEF7ED71EDF7FEFBFEF31
:10808300BFE77EDF3EE75FE77FF7DFF7DFF7DFE797
:10809300BFC6DEBE7DB65CD77FE7DFE7DFBEBDA62A
:1080A3003DB69DCF5EDF7EF79FF7BFF7DFE79FD734
:1080B3003ECF3FC71FC6DFC6FFCEFFD73EDF7EE7FB
:1080C3009EE7BFD73EBEBEAEBE9E7E9E5E9E5F9EB9
:1080D3007F9E7F9E7E9EBF9E9F9E9F9EBF9EBF96BE
:1080E3009E969E969E9EBEA6BEA6BEA6BEA6BEA6F5
:1080F300BEA6DEA6BEA6DEA6BE9E9E9E7DA6BFAE85
:10810300DFA69EA69EA6BEAEFFA6BFAEBFBEFFC69F
:10811300FECF1ECEDDC6DDCF1ECF1FD71FDF1EE76E
:108123005EE75FD73FBEFDC6DEC6DFAEFF9EBF9EE6
:108133007F967E969E8E9E8EBF8EBF8E9F96BF9697
:10814300BFA6DFB71FB6FFB6DEBEDFBEDFBEDFBE34
:10815300DEBEFFB6FEAEFFA6DF965D8E7E8E9E86EA
:108163009F869F7E9F7E9F7E9E7E9F7E7F769E7E46
:10817300BF7E7F867F8E7F969FA6BE9E9D8E9E9698
:108183009E9E9E9EBFA6BFAEDFAEFFAEFFAF1FAFEC
:108193001FB71FAEFFAEFFAEFEA6FEAEFFAF1FAE14
:1081A300FFAEFFAEFFAEFFAEDFA6FF9EFFA6DFA6CC
:1081B300BFA6DFA6BF9EBF9EBF9EBF96DF96BF8EA4
:1081C300BF86BF869E7E9E765E765F6E5F6E5E66C0
:1081D3005E663E661E6E3F6E5E6E5E6E5E767F769A
:1081E3005E765E7E7E7E5E533042AE0886426D8C46
:1081F300956BD263F36C754B921A2D32F08DBBA63F
:108203009EBEDDC6FDD75EDF5EDF3EDF3EDF3DD7D0
:108213001DC69DBE9CAE3BBEDDEFFFF7FFFFFFFF1C
:10822300FFFFDFFFFFF7FFD73EAE7DAE9F963E8E8B
:108233003F863F85FDA65DE7BFF7DFF7DFF7DEF794
:10824300DEEFDFC6DDBE7DCEDDDF1DE73EE77EE789
:10825300BFE7BFE79FEF7EF7BFF7FFF7DFF7DFEF7C
:10826300FFC6BCBE5CC6BEBE9DDF7FEFDEEFDFDFB9
:108273009FB65CAE3CAE1BB6DDC73EBEFEB6BECF00
:108283003FDFFFCF7DCEFDDF3FEF7FF7DFE79FCF00
:108293001EC6FFBEDFB6BEBEBEBEBECF3FDF7FDFA4
:1082A3009FE7BFCEFDB63B961D8E3E8E3E8E3E961D
:1082B3007F969F9EBF9EBF9EBE9EBF9EBF9EBF9E3C
:1082C300BE96BE9EDFAF1FB71FBF3FBF5FBF3FC797
:1082D3005FC75FC73FC73FC75FC75FC75FBEFEB626
:1082E300DFB6DFB6DFB71FAEDFAEDFB6FFBEDFC67A
:1082F300FEC6FEC71EC71EBEFEC6FFCF1FDF5FE75B
:108303007FDF5FC73FAEBEA65CAE9E9E7E8E7E962F
:108313007E969D969D8EBE96DE96BE969E9E9F9E53
:10832300BF96BF969F969F967E965E967F967F9604
:108333007E967E8E5E8E5E865E869F869F869F8EEF
:108343007E8E7E867E867E867E869E869F7E9E7EB1
:108353009E7E7E867E867E869E7E7D86BE86BF864A
:108363009F8EBF8EBF8E9F8EBF86BF8EBF8EDF8ECA
:108373009F969F8E7E8E5E865D7E5D865D865D8E1C
:108383009E96BE9EDF9EFF96DF96DF96DF96BF9694
:10839300BF969F9E9F9EDF9EDFAEBFAEDFAEDFA682
:1083A300DFA6DF9E9F8E7F865F765F6E5F663E668B
:1083B3003E663E663E6E1F661E663F6E5F6E7F665E
:1083C3005E665E6E5E6E3E07E007E007E007E0076D
:1083D300E007E007E007E007E007E007E007E00762
:1083E300E007E007E007E007E007E007E007E00752
:1083F300E007E007E007E007E007E007E007E00742
:10840300E007E007E007E007E007E007E007E00731
:10864300E096B6BE3A773207E007E007E007E007B7
:10865300E007E007E007E007E007E007E007E007DF
:10866300E007E007E007E007E007E007E007E007CF
:10867300E007E007E007E007E007E007E007E007BF
:10868300E007E007E007E007E007E007E007E007AF
:10869300E007E007E007E007E007E007E007E0079F
:1086A300E007E0478DB5FAADF9C61AB67967510709
:1086B300E007E007E007E007E007E007E007E0077F
:1086C300E007E007E007E007E007E007E007E0076F
:1086D300E007E007E007E007E007E007E007E0075F
:1086E300E007E007E007E007E007E007E007E0074F
:1086F300E007E007E007E007E007E007E007E0073F
:10870300E007E007E007E07EF3BDDAADF9ADF9B5C8
:10871300F9C61BAE98576F07E007E007E007E007CD
:10872300E007E007E007E007E007E007E007E0070E
:10873300E007E007E007E007E007E007E007E007FE
:10874300E007E007E007E007E007E007E007E007EE
:10875300E007E007E007E007E007E007E007E007DE
:10876300E007E007E007E007E007E0AE58B5D9AD62
:10877300D9ADD9ADD8ADF9B5D9C5FB9ED63FAD07B7
:10878300E007E007E007E007E007E007E007E007AE
:10879300E007E007E007E007E007E007E007E0079E
:1087A300E007E007E007E007E007E007E007E0078E
:1087B300E007E007E007E007E007E007E007E0077E
:1087C300E007E007E007E007E007E007E05F4FBDF1
:1087D300FAADD9B5D9B5D9ADF9ADD8CEBBC67ABD49
:1087E300B9C61A8EF42FAB07E007E007E007E007EE
:1087F300E007E007E007E007E007E007E007E0073E
:10880300E007E007E007E007E007E007E007E0072D
:10881300E007E007E007E007E007E007E007E0071D
:10882300E007E007E007E007E007E007E007E0070D
:10883300E08EB5B5DAADF9ADD9ADD9B5F9ADD8D6C8
:10884300BBF7DFE73CBE19BDDAB6597F1207E00775
:10885300E007E007E007E007E007E007E007E007DD
:10886300E007E007E007E007E007E007E007E007CD
:10887300E007E007E007E007E007E007E007E007BD
:10888300E007E007E007E007E007E007E007E007AD
:10889300E007E03FACBE19ADD9B5D9ADD9ADD9AD7F
:1088A300D9ADD9ADB8BE19E73DFFDFD6FCB5F9C5E3
:1088B300FBBE796F5107E007E007E007E007E00739
:1088C300E007E007E007E007E007E007E007E0076D
:1088D300E007E007E007E007E007E007E007E0075D
:1088E300E007E007E007E007E007E007E007E0074D
:1088F300E007E007E007E07712BDDAADD8ADD9AD08
:10890300D9ADD9ADD9ADD9ADF9ADD8ADB8C65ADF6A
:108913001CADF9ADF9B5FAC61BAE98478D07E00754
:10892300E007E007E007E007E007E007E007E0070C
:10893300E007E007E007E007E007E007E007E007FC
:10894300E007E007E007E007E007E007E007E007EC
:10895300E007E007E007E007E007E0A657B5D9AD79
:10896300F8ADD9ADD9ADD9ADD9ADD9ADD9ADF9AD95
:10897300F9ADD8ADB8ADD9ADD9ADD9ADF9BDFAAE74
:108983003807E007E007E007E007E007E007E00754
:10899300E007E007E007E007E007E007E007E0079C
:1089A300E007E007E007E007E007E007E007E0078C
:1089B300E007E007E007E007E007E007E0576FBDE7
:1089C300DAADD9ADF8ADD9ADD9ADD9ADD9ADD9AD54
:1089D300D9ADD9ADD9B5F9B5F9ADD9ADD9ADD9AD14
:1089E300F8AD98963507E007E007E007E007E007F2
:1089F300E037A96EC907E007E037A907E007E007FA
:108A0300E007E007E007E007E007E007E007E0072B
:108A1300E007E007E007E007E007E007E007E0071B
:108A2300E08EB4BDDAADF9ADD8ADD9ADD9ADD9AD20
:108A3300D9ADD9ADD9ADD9ADD9ADD9ADD9ADD9AD03
:108A4300D9ADD9ADD8B5785F0F07E007E007E007E8
:108A5300E007E007E0CE248E4707E0966607E007CD
:108A6300E007E007E007E007E007E007E007E007CB
:108A7300E007E007E007E007E007E007E007E007BB
:108A8300E007E037ACB619ADD9ADF9B5D9ADD9AD7D
:108A9300D9ADD9ADD9ADD9ADD9ADD9ADD9ADD9ADA3
:108AA300D9ADD9ADD9ADF9ADB8ADD707E007E0077A
:108AB300E007E007E05F0907E0BD649CA56728F5D0
:108AC300025E8807E007E007E007E007E007E0074A
:108AD300E007E007E007E007E007E007E007E0075B
:108AE300E007E007E007E06F11BDDAADF8ADD9ADFF
:108AF300D9ADD9ADD9ADD9ADD9ADD9ADD9ADD9AD43
:108B0300D9ADD9ADD9ADD9ADD9ADF9B5797E930785
:108B1300E007E007E007E09EA68E6707E075C80759
:108B2300E04749AC6436C807E007E007E007E00721
:108B3300E007E007E007E007E007E007E007E007FA
:108B4300E007E007E007E007E007E0A677B5DAAD66
:108B5300D9ADD9ADD9ADD9ADD9ADD9ADD9ADD9ADE2
:108B6300D9ADD9ADD9ADD9ADD9ADD9ADD9ADD8ADD3
:108B730098476D07E007E007E007E0C5C5CC63074A
:108B8300E007E007E0470907E007E007E007E00741
:108B9300E007E007E007E007E007E007E007E0079A
:108BA300E007E007E007E007E007E007E0476DBD07
:108BB300FAADF9ADD9ADD9ADD9ADD9ADD9ADD9AD41
:108BC300D9ADD9ADD9ADD9ADD9ADD9ADD9ADD9AD72
:108BD300F9AD989E3607E007E007E03FA907E08577
:108BE300A83E6807E0A685AE0607E007E007E007B2
:108BF300E007E007E007E007E007E007E007E0073A
:108C0300E007E007E007E007E007E007E007E00729
:108C1300E086D4BDDAADD8ADD9ADD9ADD9ADD9AD36
:108C2300D9ADD9ADD9ADD9ADD9ADD9ADD9ADD9AD11
:108C3300D9B5D9ADF9B57966F007E007E05F476EBE
:108C4300A807E0378A07E007E0A606CC2307E0077A
:108C5300E007E007E007E007E007E007E007E007D9
:108C6300E007E007E007E007E007E007E007E007C9
:108C7300E007E02FCBB618ADD9ADF9B5D9B5D9B565
:108C8300D8B5D8B5D8ADD8ADD8ADD8ADD8ADD8ADA9
:108C9300D8ADD8ADD8B5D8ADD8ADD737AB07E00789
:108CA300E0DDE4B58507E007E066E82FAA6E082E4D
:108CB300E907E007E007E007E007E007E007E00770
:108CC300E007E007E007E007E007E007E007E00769
:108CD300E007E007E007E06F11BDDAADD8ADD8B526
:108CE300D8B5D8B5B8B5D8B5B8ADD8ADD8ADD8AD79
:108CF300D8ADD8ADD8ADD8ADD8ADD8B59886930793
:108D0300E007E007E0A5667D0507E06F27CDC40710
:108D1300E007E007E007E007E007E007E007E00718
:108D2300E007E007E007E007E007E007E007E00708
:108D3300E007E007E007E007E007E09E56B5D9AD9E
:108D4300D8ADD8ADD8ADD8ADD8B5D8B5D8ADD8ADE8
:108D5300D8ADD8ADD8ADD8ADD8ADD8ADD8ADD8B5E0
:108D630078574E07E007E0378A5EAA07E007E07608
:108D7300E8E4024E8907E007E007E007E007E007C1
:108D8300E007E007E007E007E007E007E007E007A8
:108D9300E007E007E007E007E007E007E0478DBDF5
:108DA300F9ADF9B5D9ADD9ADD9ADD9ADF9ADF9AD08
:108DB300F8ADD9ADD9ADD9ADD9B5F9ADD9ADD9AD39
:108DC300F8ADB895F507E007E007E007E007E0072F
:108DD300E007E06689560807E007E007E007E007D9
:108DE300E007E007E007E007E007E007E007E00748
:108DF300E007E007E007E007E007E007E007E00738
:108E0300E08ED4BDDAA5B8ADB8B5F9ADD9ADD9B555
:108E1300F9B5F9ADD9ADD9ADD9ADD9ADD9ADD9ADD7
:108E2300D9ADD9ADD9B5796EF107E007E007E00711
:108E3300E007E007E007E02F8A07E007E007E00725
:108E4300E007E007E007E007E007E007E007E007E7
:108E5300E007E007E007E007E007E007E007E007D7
:108E6300E007E007E0AE38B5D98CB4A577B5F9AD26
:108E7300D9ADD9B5D9B5D9B5D9ADD9ADD9ADD9ADA7
:108E8300D9ADD9ADD9ADD9ADD9ADB837AC07E007B8
:108E9300E007E007E007E007E007E007E007E00797
:108EA300E007E007E007E007E007E007E007E00787
:108EB300E007E007E007E007E007E007E007E00777
:108EC300E007E007E007E05F30C5DAADD894D5B539
:108ED300D9ADD9ADD9ADD9ADD9ADD9ADD9ADD9AD5F
:108EE300D9ADD9ADD9ADD9ADD9ADF9B59986740799
:108EF300E007E007E007E007E007E007E007E00737
:108F0300E007E007E007E007E007E007E007E00726
:108F1300E007E007E007E007E007E007E007E00716
:108F2300E007E007E007E007E007E09E96B5FAA553
:108F330077A577B5F9ADD9ADD9ADD9ADD9ADD9ADA2
:108F4300D9ADD9ADD9ADD9ADD9ADD9ADD9ADD8B5E7
:108F530098574F07E007E007E007E007E007E0075F
:108F6300E007E007E007E007E007E007E007E007C6
:108F7300E007E007E007E007E007E007E007E007B6
:108F8300E007E007E007E007E007E007E03F8DBD0B
:108F9300FAADF98CD4ADB8B5F9ADD9ADD9ADD9AD7C
:108FA300D9ADD9ADD9ADD9ADD9ADD9ADD9ADD9AD8E
:108FB300F9ADB9A5F607E007E007E007E007E0072A
:108FC300E007E007E007E007E007E007E007E00766
:108FD300E007E007E007E007E007E007E007E00756
:108FE300E007E007E007E007E007E007E007E00746
:108FF300E07EF3BDDAA59794F5B5F9ADD9ADD9AD5A
:10900300D9ADD9ADD9ADD9ADD9ADD9ADD9ADD9AD2D
:10901300D9ADD9ADF9B57976D207E007E007E00716
:10902300E007E007E007E007E007E007E007E00705
:10903300E007E007E007E007E007E007E007E007F5
:10904300E007E007E007E007E007E007E007E007E5
:10905300E007E007E0A637B5F994F5A577B5F9ADD4
:10906300D9ADD9ADD9ADD9ADD9ADD9ADD9ADD9ADCD
:10907300D9ADD9ADD9ADF9ADB8ADB73F8C07E007E0
:10908300E007E007E007E007E007E007E007E007A5
:10909300E007E007E007E007E007E007E007E00795
:1090A300E007E007E007E007E007E007E007E00785
:1090B300E007E007E007E05F4FBDDAA5B78CB4AD8A
:1090C300D8B5F9ADD9ADD9ADD9ADD9ADD9ADD9AD46
:1090D300D9ADD9ADD9ADD9ADD9ADF9B5998E5407BF
:1090E300E007E007E007E007E007E007E007E00745
:1090F300E007E007E007E007E007E007E007E00735
:10910300E007E007E007E007E007E007E007E00724
:10911300E007E007E007E007E007E08E95B5DAAD8A
:10912300D8A577B5F9ADD9ADD9ADD9ADD9ADD9AD4F
:10913300D9ADD9ADD9ADD9ADD9ADD9ADD9ADD8B5F5
:10914300785F2F07E007E007E007E007E007E007A5
:10915300E007E007E007E007E007E007E007E007D4
:10916300E007E007E007E007E007E007E007E007C4
:10917300E007E007E007E007E007E007E007E08E2D
:1091830074B519ADB8ADF9ADD9ADD9ADD9ADD9ADCA
:10919300D9ADD9ADD9ADD9ADD9ADD9ADD9ADD9AD9C
:1091A300F9B5B99DD607E007E007E007E007E00758
:1091B300E007E007E007E007E007E007E007E00774
:1091C300E007E007E007E007E007E007E007E00764
:1091D300E007E007E007E007E007E007E007E00754
:1091E300E007E007E06EB1A577AD38ADB8ADF9ADF6
:1091F300D9ADD9ADD9ADD9ADD9ADD9ADD9ADD9AD3C
:10920300D9ADD9ADF9B57976B207E007E007E00744
:10921300E007E007E007E007E007E007E007E00713
:10922300E007E007E007E007E007E007E007E00703
:10923300E007E007E007E007E007E007E007E007F3
:10924300E007E007E007E007E007E037AC7672AD40
:1092530057AD38ADD8B5F9B5D9ADD9ADD9ADD9ADCF
:10926300D9ADD9ADF8ADF9ADD9AD983F8D07E007CC
:10927300E007E007E007E007E007E007E007E007B3
:10928300E007E007E007E007E007E007E007E007A3
:10929300E007E007E007E007E007E007E007E00793
:1092A300E007E007E007E007E007E007E007E00783
:1092B300E007E0476D8E14AD37AD77ADD8B5F9ADA6
:1092C300D9ADD9ADD9ADD9ADF8ADF9B599963507C5
:1092D300E007E007E007E007E007E007E007E00753
:1092E300E007E007E007E007E007E007E007E00743
:1092F300E007E007E007E007E007E007E007E00733
:10930300E007E007E007E007E007E007E007E00722
:10931300E007E007E007E007E007E0574E9DD5AD23
:1093230037A598ADF9B5F9ADD9ADD9ADF8ADF9B566
:1093330079673007E007E007E007E007E007E007A9
:10934300E007E007E007E007E007E007E007E007E2
:10935300E007E007E007E007E007E007E007E007D2
:10936300E007E007E007E007E007E007E007E007C2
:10937300E007E007E007E007E007E007E007E007B2
:10938300E007E067119DB6AD38AD98ADF8B5F9AD1E
:10939300F8ADB8A5D707E007E007E007E007E00767
:1093A300E007E007E007E007E007E007E007E00782
:1093B300E007E007E007E007E007E007E007E00772
:1093C300E007E007E007E007E007E007E007E00762
:1093D300E007E007E007E007E007E007E007E00752
:1093E300E007E007E007E007E007E07EB3A576AD1E
:1093F30038A5B8ADF8AD7876B207E007E007E00727
:10940300E007E007E007E007E007E007E007E00721
:10941300E007E007E007E007E007E007E007E00711
:10942300E007E007E007E007E007E007E007E00701
:10943300E007E007E007E007E007E007E007E007F1
:10944300E007E007E007E007E007E007E007E007E1
:10945300E037AB7692A577AD37AD77378C07E0076A
:10946300E007E007E007E007E007E007E007E007C1
:10947300E007E007E007E007E007E007E007E007B1
:10948300E007E007E007E007E007E007E007E007A1
:10949300E007E007E007E007E007E007E007E00791
:1094A300E007E007E007E007E007E007E007E00781
:1094B300E007E007E007E007E03FAC7E92671007B4
:1094C300E007E007E007E007E007E007E007E00761
:1094D300E007E007E007E007E007E007E007E00751
:1094E300E007E007E007E007E007E007E007E00741
:1094F300E007E007E007E007E007E007E007E00731
:10974300E007E007E007E007E007E007E007E0FFE6
:10975300DFFFDFFFDFFFDFFFDFFFDFFFDFFFDFFF16
:10976300DFFFDFFFDFF7BEFFDFFFDFFFDFFFDFFF2F
:10977300DFFFDFFFDFFFDFFFDFFFDFFFDFFFDFFFF6
:10978300DFFFDFFFDFFFDFFFDFFFDFFFDFFFDFFFE6
:10979300DFFFDFFFDFFFDFFFDFFFDFFFDFFFDFFFD6
:1097A300DFFFDFFFDFF7BEF7DFF7DFF7DFF7BEF738
:1097B300BFF7BEF7BFF7BFF7BEF7DFF7BEFFDFFFA9
:1097C300BEFFDFFFDFFFDFFFDFFFDFFFDFFFDFFFC7
:1097D300DFFFDFFFDFFFDFFFDFFFDFF7BEF7BEF7F0
:1097E300BEF7BEF7BEF7BEF7BFF7BEF7BEF7BEFFC5
:1097F300DFF7BEFFDFFFDFFFDFFFDFFFDFFFDFFF9F
:10980300DFFFDFFFDFFFDFFFDFFFDFFFDFFFDFFF65
:10981300DFF7BEFFDFFFDFFFDFFFDFFFDFFFDFFF7E
:10982300DFFFDFF7BEFFDFFFDFFFDFFFDFFFDFFF6E
:10983300DFFFDFFFDFFFDFFFDFFFDFFFDFFFDFFF35
:10984300DFFFDFFFDFFFDFFFDFFFDFFFDFFFDFFF25
:10985300DFFFDFFFDFFFDFFFDFFFDFFFDFF7BEFF3E
:10986300DFFFDFFFDFFFDFFFDFFFDFFFDFFFDFFF05
:10987300DFFFDFFFDFFFDFFFDFFFDFF7BEFFDFFF1E
:10988300DFFFDFF7DFF7DFF7DEF7DFF7BEF7DFFF37
:10989300DFFFDFFFDFFFDFFFFFFFFFFFFFFFFFFF55
:1098A300FFFFFFFFFFFFFFFFFFFFFFFFFFFFFFFFC5
:1098B300DFF7DFF7DEEFDEEFBEE7BEE7BEE7BEE7CB
:1098C300BFEFDEF7DFFFFFFFFFFFFFFFFFFFFFFF3E
:1098D300FFFFFFFFFFFFFFFFFFFFFFFFFFFFFFFF95
:1098E300FFFFFFFFFFFFDFFFDFFFDFFFDFF7DFF735
:1098F300BEF7DFF7BEFFDFFFDFFFDFFFDFFFDFFFC7
:10990300DFFFDFFFDFFFDFFFDFF7BEFFDFFFDFFF8D
:10991300DFFFFFFFDFFFDFFFDFFFDFFFDFFFDFFF34
:10992300DFFFDFFFDFFFDFFFDFFFDFFFDFFFDFFF44
:10993300DFFFDFF7BEFFDFFFDFFFDFF7BEFFDFFF86
:10994300DFFFDFFFDFFFDFFFDFFFDFFFDFFFDFFF24
:10995300DFFFDFFFDFFFDFFFDFFFDFFFDFFFDFFF14
:10996300DFFFDFFFDFFFDFFFDFF7BEF7DFF7DFFF3D
:10997300DFFFDFFFFFFFFFFFFFFFFFFFFFFFFFFF34
:10998300FFF7DFDFBFCF7EC73EAEDD9E7C9E1B8D24
:10999300DB6D5964F85CB85C7754574C363C172B35
:1099A30095237523351B341B351AF412F51AD31B73
:1099B300141AF4231423142B3433553B5543B64B59
:1099C300B553B653F6649885198D598DBAAE1BBE3F
:1099D3007CC6FDE77EF7BEFFFFFFFFFFFFFFFFFF34
:1099E300FFFFFFFFFFFFDFFFDFFFDFFFDFFFDFFF24
:1099F300DFFFDFFFDFFFDFFFDFFFDFFFDFFFDFFF74
:109A0300DFFFDFF7BEFFDFFFDFFFDFFFDFFFDFFF8C
:109A1300DFFFDFFFDFFFDFFFDFFFDFFFDFFFDFFF53
:109A2300DFFFDFF7BEFFDFFFDFFFDFFFDFFFDFFF6C
:109A3300DFFFDFFFDFFFDFFFDFF7BEFFDFFFDFF764
:109A4300BEFFDFFFDFFFDFF7BEFFDFFFDFF7DFF77D
:109A5300DFF7BFF7BFFFBFFFDFFFFFFFFFFFFFFF23
:109A6300FFF7DFD79EC73DA6BC8E9C65FA65BA4556
:109A7300792CD814570BD603B60355035502D403D8
:109A83001502F402F402B4029302D4027302D40264
:109A93007302B402730253025301F2021201B102C0
:109AA3001201F202530A7312931AB41AF423753390
:109AB3005543754B7553954BB54395439543954323
:109AC300B53BD643B753B66CB864B86D398E3BAE6D
:109AD3009CC71DDF5EEFBFFFBEFFDFFFDFFFDFFFC2
:109AE300DFFFDFFFDFFFDFFFDFFFDFFFDFFFDFFF83
:109AF300DFFFDFF7BEFFDFFFDFFFDFFFDFFFDFFF9C
:109B0300DFFFDFFFDFFFDFFFDFFFDFFFDFFFDFFF62
:109B1300DFFFDFFFDFFFDFFFDFFFDFFFDFFFDFFF52
:109B2300DFFFDFFFDFFFDFFFDFFFDFFFDFFFDFFF42
:109B3300DFFFDFFFDFFFDFF7DFF7DFFFDFFFDFFF42
:109B4300FFFFFFFFFFFFFFDF9EB71D8E9C5DDA4522
:109B5300993D592D39457A3D79359A24F80CF90404
:109B630057041703F603D603F70395041703950366
:109B7300B60375037503950375037502D4031502C4
:109B83009302D40AF413552BD65C576CF98DBA9E05
:109B93003CBEBDD71EE7BFEFDFF7DFFFFFFFFFFFD1
:109BA300FFFFFFFFFFFFFFFFFFFFFFFFFFFFFFFFC2
:109BB300FFFFFFF7DFEF7EE75ECEFDBE9CAEBC96F8
:109BC3005B9E9C965BA6BCBEBCDF3EF7BEFFDFFF81
:109BD300DFFFDFFFDFFFDFFFDFFFDFFFDFFFDFFF92
:109BE300DFFFDFFFDFFFDFFFDFFFDFFFDFFFDFFF82
:109BF300DFFFDFFFDFFFDFFFDFFFDFFFDFFFDFFF72
:109C0300DFFFDFFFDFFFDFFFDFFFDFFFDFFFDFFF61
:109C1300DFFFDFFFDFFFDFFFDFFFDFFFDFF7BEF782
:109C2300BEF7DFF7DFFFFFFFFFFFFFFFFFEFDFB74A
:109C33001D865C5DDB35191D3A351955DB7E5C9E4F
:109C4300FDCF7EEFBEEFFF6E5B2D190417041703E4
:109C5300D6041704370416043703D6041703B603D0
:109C6300F603B50376035502D403761BB644B96DE8
:109C7300799E5BC71DE7BEFFFFFFFFFFFFFFFFFFEF
:109C8300FFFFFFFFFFFFDFFFDFFFDFFFBEFFBFFFC2
:109C9300BFF7BFF7BEF7BEF7BFF7BEF7BFFFDFFFE4
:109CA300DFFFDFFFDFFFDFFFFFFFFFFFFFFFFFFF41
:109CB300FFFFFFFFFFF7DFF7BEF7BEF7BFFFDFFFD3
:109CC300DEFFDFFFDFFFDFFFDFFFDFFFDFFFDFFFA2
:109CD300DFFFDFF7BEFFDFFFDFFFDFFFDFFFDFFFBA
:109CE300DFFFDFFFDFFFDFFFDFFFDFFFDFFFDFFF81
:109CF300DFFFDFFFDFFFDFFFDFFFDFFFDFFFDFFF71
:109D0300DFFFDFFFDFFFDFFFDFFFDFFFDFFFDFFF60
:109D1300DFFFFFFFFFE7BFB6FD765B3D7915192532
:109D2300193D7A7E3CB6FDDF9EF7DFFFFFFFFFFFA5
:109D3300FFFFFFFFDFFFDFF7DFEFBEC75D8E9C4551
:109D43007A24B8043703D603F703D60457039603DC
:109D5300B603B61C3745198DFBC73EEFBEFFFFFFA9
:109D6300FFFFFFFFFFFFDFFFDFF7BEF7BFF7BEF722
:109D7300DFF7BFFFDFFFDFFFDFFFDFF7BEFFDFFF41
:109D8300DFFFDFFFDFFFDFFFDFFFDFFFDFFFDFFFE0
:109D9300DFFFDFFFDFF7BFFFDFFFDFF7BFF7BFF750
:109DA300BEF7DFFFDFFFDFFFDFFFDFFFDFFFDFFFE9
:109DB300DFFFDFFFDFFFDFFFDFF7BEFFDFFFDFFFD9
:109DC300DFFFDFFFDFFFDFFFDFFFDFFFDFFFDFFFA0
:109DD300DFFFDFFFDFFFDFFFDFFFDFFFDFFFDFFF90
:109DE300DFFFDFF7DFFFDFFFDFFFDFFFDFF7DEFF91
:109DF300DFFFDFFFDFFFBEFFDFFFDFFFDFFFDFD7B9
:109E03009E7EDC3DBA25191CB83D9A7E5BBF3DEFB3
:109E1300BFFFFFFFFFFFFFFFDFF7BEF7BFF7DFF770
:109E2300DFF7BEFFDFFFDFFFDFFFDFFFFFFFFFFF28
:109E3300FFE7BEC73D8E5B4D5A1C770C58247875DF
:109E4300DBB6FDE79EFFFFFFFFFFFFFFDFF7BEF778
:109E5300BEF7DFFFDFF7DFFFDFFFDFFFDFFFDFFF40
:109E6300DFF7BEFFDFFFDFFFDFFFDFFFDFFFDFFF28
:109E7300DFFFDFFFDFFFDFFFDFFFDFFFDFF7BEFF18
:109E8300DFFFDFFFDFF7BEFFDFFFDFFFDFFFDFFF08
:109E9300DFFFDFFFDFFFDFFFBFFFBFFFDFFFDFFF0F
:109EA300DFFFDFFFDFFFDFFFDFF7BEFFDFFFDFFFE8
:109EB300DFFFDFFFDFFFDFFFDFFFDFFFDFFFDFFFAF
:109EC300DFFFDFFFDFFFDFFFDFFFDFFFDFFFDFF7A7
:109ED300DFF7DFFFDFFFDFF7BEF7BEF7BEF7BEF743
:109EE300BEF7BEFFDFFFDFFFDFF7BEF7BEFFBEC774
:109EF3003D8EDC96BCBF1DE7BEFFFFFFFFFFFFFFEC
:109F0300BEFFBEF7BEF7BFFFDFF7DFFFDFFFFFFFD9
:109F1300DFFFDFF7BEFFBEFFDFF7DFF7BEF7BEF7FA
:109F2300BEFFBEFFDFFFFFFFFFE79ECF5DF7FFFF33
:109F3300FFFFFFFFDFF7BEF7DFF7BEF7BEF7BEF7A2
:109F4300BEF7BEFFDFF7BEF7BEF7BEF7BEF7BEF73D
:109F5300BEF7BEF7BEF7BEFFDFFFDFF7BEF7BEF704
:109F6300BEF7BEF7BEF7BEF7BEF7BEF7BEF7BEF746
:109F7300BEF7BEF7BEFFDFFFDFFFDFFFDFFFDFF769
:109F8300BEF7BEF7BEFFDFF7BEFFDFFFDFFFFFFF5A
:109F9300FFFFDFFFDFFFDFFFDFFFDFFFDFF7BEF7DF
:109FA300BEF7BEF7BEF7BEF7BEF7BEFFDFF7BEFFD5
:109FB300DFF7BEF7BEF7BEFFDFFFDFFFDFFFDFFF29
:109FC300DFFFDFFFDFFFDFFFFFFFFFFFFFFFFFFF1E
:109FD300FFFFFFFFDFF7BEF7BEFFFFFFFFFFFFFF40
:109FE300FFFFFFFFFFFFFFFFFFF7BEF7DFF7FFFFF7
:109FF300FFFFFFFFFFFFFFFFFFFFDFFFBEFFBEFF10
:10A003009EFFDFFFFFFFFFFFDFFFFFFFFFFFFFFFFE
:10A01300FFFFFFFFFFF7DFF7DFFFFFFFFFFFDFF7C5
:10A02300DFFFFFFFFFFFFFFFDFFFFFFFFFFFFFFF7D
:10A03300FFFFFFFFFFFFFFFFFFFFFFFFFFFFFFFF2D
:10A04300FFFFFFFFFFFFFFFFDFFFFFFFFFFFFFFF3D
:10A05300FFFFFFFFFFFFFFFFFFFFFFFFFFFFFFFF0D
:10A06300FFFFFFFFFFFFDFFFDFFFDFF7BEFFFFFFA6
:10A07300FFFFFFFFFFFFFFFFFFFFFFF7BEF79EF7A7
:10A083009EF7BEFFDFFFFFFFFFFFDFFFDFFFFFFFE7
:10A09300FFFFFFFFFFFFFFFFFFFFFFFFFFFFFFFFCD
:10A0A300FFFFFFFFFFFFFFFFDFFFDFFFDFFFDFFF3D
:10A0B300DFFFDFF7BEFFDF8430630C632C632C7399
:10A0C3008EAD55F79EFFFFFFFFD69A8410630C6396
:10A0D3000C5B0C634DDEFBFFDFFFFFFFFFFE59FC54
:10A0E300B2FB4DFACBF9C7F924F924F9A6FA08FA19
:10A0F30049FA69FA69FAEBFF1CE75D6B6D630C6360
:10A103000C630C9CF3FFFFFFDFFFDFFFDFFFDFFFCD
:10A11300FFAD75630C9CD3FFFFDEDB632C630C6325
:10A123000C630C5AEB528A4A694A69528A4A695249
:10A133008A528A528AB596FFDFEF5D6B6D630C63BB
:10A143000C630C5AEB528A528A528A528A528A5AA6
:10A15300CB8410B5B6FFDFFFDFFFDFFFFFE73CB5C2
:10A16300968410630C4A6931862124296542084A82
:10A1730049528A528A528A9492FFDFFFFFBDF78CBD
:10A18300516B4D630C52AA4A694A494A494A494AA2
:10A1930069528A7BEFD69AFFFFFFDFFFDFFFDFFF06
:10A1A300DFFFDFF7BEFFFF31860000000000000085
:10A1B30000000029658C515ACB000000000000000C
:10A1C3000000000000AD55FFFFF659F9E7F841F82C
:10A1D30000F800F800FAAAFD14FE59FEBAFEFBFFD0
:10A1E3001CFEBAFE59FE18FFBEBDF70000000000BA
:10A1F30000000031A6FFFFF7BEFFDFFFDFF7BEFF62
:10A20300FF4A4900003186FFFFB5960000000000B9
:10A2130000000010A2AD55B5B6B5B6B5B6BDD7B5FD
:10A22300B6B5B6B5B6DEDBFFFFC61800000000000A
:10A2330000000010A29CD3A534A534A534A5148C2A
:10A2430071210400006B6DFFFFFFDF7BEF18C3007C
:10A25300000000000010A28410BDD7D6BAEF7DF72E
:10A263009EEF7DDEFBCE79D6BAFFFF7BCF000000E9
:10A2730000000000006B6DB596BDD7BDD7B5B6B570
:10A28300B67BEF00000861D69AFFDFF7BEFFDFFF62
:10A29300DFFFDFF7BEFFFF42080000630C632C08FB
:10A2A3004100000000000008418430420800000023
:10A2B3002000200000B5B6FF7DF0E3F800F800F8B9
:10A2C30020F800FC51FFFFFFFFFFFFFFFFFFFFFF31
:10A2D300FFFFFFFFFFF7FFFFFFBDF70000002000B8
:10A2E3002000004208FFFFF7BEFFDFFFDFF7BEFFDE
:10A2F300FF528A00004208FFFFBDD7000000200084
:10A3030020000018E394B29CF39CF39CF39CF39C11
:10A31300F39CF3CE59FFFFFFFFC638000000200077
:10A323002000004228FFFFFFFFFFFFFFFFFFFFFFAB
:10A33300FF8C5100002945FFFF8C710000000000D5
:10A3430020002018E3E71CFFFFFFFFEF7DD69AD61E
:10A353009AD69ADEFBE73CFFDFFFFF31A600000041
:10A363002000200000738E9492949294929492947D
:10A37300927BCF00200000B5B6FFFFF7BEFFDFFFE3
:10A38300DFFFDFF7BEFFFF42080000AD55FFFFCE42
:10A393007994926B6D94B2E71CFFFF5AEB000000B7
:10A3A3000000000000B5F7FE9AF000F820F800F86E
:10A3B30000F800FE79FFFFFF9EFFBEFFBEFFBEFF5A
:10A3C300BEFFBEFFBEF79EFFFFBDF70000002000EB
:10A3D3000000004208FFDFF79EF7BEF7BEF79EFFBF
:10A3E300DF528A000039E7FFFFBDD70000000000FD
:10A3F30000000000204A695ACB5ACB5ACB5ACB5A99
:10A40300CB5ACB8410FFDFFFFFC6380000000000EB
:10A41300000000084152AA632C630C630C5AEB4AF8
:10A423006908412965A534FFFF4228000000200088
:10A433002000004228FFFFF79EF7BE843039C7395A
:10A44300C73186086100004A69FFFF420800000027
:10A4530000000000004208738E738E738E738E7338
:10A463008E4A4900000000BDF7FFFFFFDFFFDFFF5B
:10A47300DFFFDFF7BEFFFF420800009CD3FFDFFFD3
:10A48300FFFFFFFFFFFFFFFFFFFFDF528A00000018
:10A493002000200000B575FFDFFA69F800F800F826
:10A4A30000F800FA8AFF3CFFFFFFFFFFFFFFFFFFFB
:10A4B300FFFFFFFFFFF7FFFFFFBDF70000000000F6
:10A4C3000000004208FFFFFFFFFFFFFFFFFFFFFF4A
:10A4D300FF528A000039E7FFFFBDD70000000000EC
:10A4E30000000039C7FFFFFFFFFFFFFFFFFFFFFF74
:10A4F300FFFFFFFFFFF7BEFFFFCE59000000000084
:10A5030000000018E38C518C718C518C518C71A517
:10A5130034CE79F79EFFFFFFFFBDF7002000000058
:10A523000000001082BDF7FFFFFFFFFFFFFFFFFFEB
:10A53300FFFFFF5ACB000039C7FFFF39E7000000D8
:10A543002000200000CE59FFFFFFFFFFFFFFFFFFAA
:10A55300FFD6BA00000000BDF7FFFFF7BEFFDFFF25
:10A56300DFFFDFF7BEFFFF318600009CF3FFFFF73D
:10A57300BEF7BEF7BEF7BEF7BEFFFF52AA0000004C
:10A583000000000000B5B6FFFFF79EFC51F986F806
:10A5930082F800F800F841FA28FBCFFC92FC92FC09
:10A5A30092FC71FC51FC10FF1CEF7D630C10A200A8
:10A5B300200000000042085ACB5AEB5AEB5AEB42F8
:10A5C300280000000039E7FFFFEF7D738E210408A8
:10A5D30041000031A6FFDFF7BEF7BEF7BEF7BEF7B7
:10A5E300BEF7BEF7BEFFDFFFDFF7BE738E18C300F3
:10A5F30000000039E7FFFFFFFFFFFFFFFFFFFFFF43
:10A60300FFFFFFFFDFF7BEFFDFFFFFC6385ACB18A0
:10A61300E30841000000004A698C7194B294B2943B
:10A62300928C511082000031A6FFFF39C700000051
:10A633000000000000BDD7FFDFF79EF7BEF79EFFC7
:10A64300DFC63800000000BDD7FFFFFFDFFFDFFFDD
:10A65300DFFFDFFFDFFFDFBDD7A534EF7DFFDFFFC8
:10A66300DFFFDFFFDFFFDFFFDFFFDFDEDB9CF39CCE
:10A67300F39CF3AD55F79EFFDFFFDFFFFFFFDFFE28
:10A68300BAFDD7FCF3FC51FB4DFAEBFAEBFAEBFB0B
:10A693000CFBAEFC30FCD3FF7DFFFFFFFFDEFBC6F0
:10A6A30018A5349CF38C718C718C718C718C718CAA
:10A6B300719CF3A534D69AFFDFFFDFFFFFEF5DCE7A
:10A6C30059AD75CE79FFDFFFDFFFDFFFDFFFDFFF70
:10A6D300DFFFDFFFDFFFDFFFDFFFDFFFFFE71CBD84
:10A6E300F79CF3D69AF7BEF7BEF7BEF7BEF7BEFFE9
:10A6F300DFF7BEFFDFFFDFFFDFFFDFFFFFFFFFEF60
:10A703005DC638AD559CD373AE630C5ACB5ACB5A46
:10A71300EB6B4D84309CD3CE59FFDFCE79A5149CCF
:10A72300F39CF3AD75F79EFFDFFFDFFFDFFFDFFF76
:10A73300DFF7BEB596AD55EF7DFFDFFFDFFFDFFF30
:10A74300DFFFDFFFDFFFDFFFFFFFFFFFFFFFDFFFB6
:10A75300DFFFDFFFDFFFDFFFDFFFDFFFFFFFFFFFC6
:10A76300FFFFFFFFFFFFFFFFDFFFDFFFBEFFDFFF97
:10A77300FFFFFFFFFFFFFFFFFFFFFFFFFFFFFFFFE6
:10A78300FFFFFFFFFFFFFFFFFFFFDFF7BEFFFFFF3F
:10A79300FFFFFFFFFFFFFFFFFFFFFFFFFFFFFFFFC6
:10A7A300FFFFFFFFFFFFFFFFDFFFDFF7BEFFFFFF3F
:10A7B300FFFFFFFFFFFFDFFFDFFFDFFFDFFFDFFF46
:10A7C300DFFFDFFFFFFFDFFFDFFFDFF7BEFFFFFF7F
:10A7D300FFFFFFFFFFFFDFFFDFFFDFFFDFFFFFFF06
:10A7E300FFFFDFFFDFFFDFFFDFFFDFFFDFFFDFFF56
:10A7F300FFFFFFFFFFFFFFFFFFFFFFFFFFFFFFFF66
:10A80300FFFFFFFFFFFFFFFFFFFFDFFFFFFFFFFF75
:10A81300FFFFFFFFFFFFFFFFDFFFDFFFDFFFDFFFC5
:10A82300DFFFDFFFFFFFFFFFFFFFDFFFDFFFDFFFD5
:10A83300DFFFDFFFDFFFDFF7BEF7BEFFDFFFDFFF77
:10A84300DFFFDFFFDFFFDFFFDFFFDFFFDFF7BEF746
:10A85300BEF7BEF7BEFFDFFFDFFFDFFFDFFFDFFF78
:10A86300DFFFBEFFBEFFBEFFBEFFBEFFBEFFBEFFDC
:10A87300BEFFBEFFBEFFBEFFDFFFDFFFDFFFDFF771
:10A88300BEF7BEF7BEF7BEF7BEF7BEF7BEF7BEF71D
:10A89300BEF7BEF7BEFFDFFFDFFFDFFFDFFFDFFF38
:10A8A300DFF7BEF7BEFFDFFFDFFFDFFFDFFFDFFF07
:10A8B300DFFFDFFFDFFFDFFFDFFFDFFFDFFFDFFFA5
:10A8C300DFF7BEF7BEFFDFFFDFFFDFFFDFFFDFFFE7
:10A8D300DFFFDFFFDFFFDFFFDFFFDFFFDFFFDFFF85
:10A8E300DFFFDFF7BEF7BEF7BEF7BEF7BEFFDFF74A
:10A8F300BEF7BEF7BEF7BEFFDFFFDFFFDFF7BEF732
:10A90300BEF7BEF7BEFFDFFFDFFFDFFFDFFFDFFFC7
:10A91300DFFFDFF7BEF7BEFFDFFFDFFFDFFFDFFF96
:10A92300DFFFDFFFDFFFDFFFDFFFDFFFDFFFDFFF34
:10A93300DFFFDFFFDFFFDFFFDFFFDFFFDFFFDFFF24
:10A94300DFFFDFFFDFFFDFFFDFFFDFFFDFFFDFFF14
:10A95300DFFFDFFFDFFFDFFFDFFFDFFFDFFFFFFFE4
:10A96300DFFFDFFFDFFFDFFFDFFFDFFFDFFFDFFFF4
:10A97300DFFFDFFFDFFFDFFFDFFFDFFFDFFFDFFFE4
:10A98300DFFFDFFFDFFFDFFFDFFFDFFFDFFFDFFFD4
:10A99300DFFFDFFFFFFFDFFFDFFFDFFFDFFFDFFFA4
:10A9A300DFFFDFFFDFFFDFFFDFFFDFFFDFFFDFFFB4
:10A9B300DFFFDFFFDFFFDFFFDFFFDFFFDFFFDFFFA4
:10A9C300DFFFDFFFDFFFDFFFDFFFDFFFDFFFDFFF94
:10A9D300DFFFDFFFDFFFFFFFDFFFDFFFDFFFDFFF64
:10A9E300DFFFDFFFDFFFDFFFDFFFDFFFDFFFDFFF74
:10A9F300DFFFDFFFDFFFDFFFDFFFDFFFDFFFDFFF64
:10AA0300DFFFDFFFDFFFDFFFDFFFDFFFFFFFDFBD75
:10AA130059A474E679E697D5D2EE95E635E5F5EED9
:10AA230057FED8EE75EE74FF17F6D7ACD1A470B409
:10AA3300F2B512A4B0942EACD1A470A491A4719CCD
:10AA430091A492ACD3A4B3A493A4B3ACF5A4B4A43B
:10AA5300B5A4D6ACF69C94949394D48C928C937CAA
:10AA6300527C737433849684D88CD974379D5B95E8
:10AA7300178CD595168CF58CD5951694D68CB594E4
:10AA8300B69CF79CB79CD7ACB7CD99D6176AA7628B
:10AA930065EE95DDF46A268B2AE5F5EE34B4CEC572
:10AAA30030E6969C0E49A5ACB0BD526AC949C58330
:10AAB300ADB5137B4C5A286AEB9430BD76BD75BD9A
:10AAC30055ACF4B515B515BD57ACF6A4B49CD48CF0
:10AAD3003173CF843184717411743284B4745484A7
:10AAE300B77C768CD9953A849574127C73741273FF
:10AAF300D16BD17BF37C33A538AD59A518AD39ACF7
:10AB0300D8B4F6E679CDB3C571FEF6D5928B2A9B00
:10AB1300CCE635EE75C550CD71EE96AC9072C99CFE
:10AB23002FC573940E6AC97B6C9C707B4B6ACA8376
:10AB33008D8BCE8BCF7B6D8C109C519C718BF09445
:10AB430031943294517BAE83EF84506B6D73EE730B
:10AB5300EF74107C9384D58D177C7584B87C9684B0
:10AB6300954ACD42AC4AED5B2F428C4A6D52EE8C36
:10AB7300559CF794969CB6C57AACB6DE38E697DE5C
:10AB830034F6B5F696FEB8EE36F676EE54EE74EE7F
:10AB930095E675BD12BD53B512B512B5328BCD9482
:10ABA3000EACF1ACF283AD942FACF2BD74B55494FA
:10ABB30050B534CDD6C5D6A492A4D3734C6B2BA574
:10ABC30012B594AD94CEB8A5948CD25B6D7C72848F
:10ABD300D584B57C969D7963D1532E4AED42AC4A18
:10ABE300AD63705AEF4A6D8414AD79AD59AD39AC8C
:10ABF300B7B4D6DE58E697E654FEF6F696E615F6B3
:10AC030077EE56EE54F6B5F6D6E696BD12BD33BDD5
:10AC130053A4B09C4F72EA940EC5B4C59483ADACF3
:10AC2300F1C5D5CE16CDF66B0A9470AD12ACF2E633
:10AC3300B9CE1683CDB553C615948EB5B3C656E7B4
:10AC43005ACED984907C518CF484B46BF295583AE3
:10AC53004B3A4B3A6C530E3A4C52EE426C52EF5213
:10AC6300AE94969CD79496C57ABD17DE38F719F63D
:10AC7300D6EE95EE56F697F657F677F695F6D6F6A0
:10AC8300D6EED7BD32A491B533A4907B6B838CB53C
:10AC930012CDD5942EA490CE15C5B4944E944E6B7C
:10ACA3000ABDB4BDB4A4F1A4B07B8BBD73CE35ADE6
:10ACB30030B572BDB3BDF3AD93C656B5F57C5095B3
:10ACC3005595358CD5A5B94ACD3A6B428C63904ADC
:10ACD300CE530F4A6D5B3063309CF7B579AD38AC1A
:10ACE300B7B4F7DE58EED8EE95EE74EE56F677F677
:10ACF30097F676F675F6D6EEB5EE96BD12A470BD50
:10AD0300538BCD6AEAACF1EED9CDD5734BB512E6D0
:10AD1300B8E6D8A4D08C2D9CAFD676B572948E8C21
:10AD23000D83CCEF19A4CF7349C5F3AD30A530AD76
:10AD330092BE35CED97C506BF07C737C738D1653E9
:10AD43004F532F530E322B426C639163303A2C7363
:10AD53009294969CD79CD7BD19BD58D617E697EE0B
:10AD630095F6B5F696F657EE57F697FEB6FEF6EE5F
:10AD7300B5EEB6BD129C50A4706AC98BCDB512D680
:10AD8300369C8F7B8BBD73D635DEB7944D62E8B5A9
:10AD930092DE96A510944D6AE8B532C5B383AB62D3
:10ADA300E783CB7B8A5AC7840C8C6FBE169D1363D3
:10ADB300AF953684B4953784B54ACE530F4ACE6BDC
:10ADC300914ACE635073D39CF8A538A519AD59ACFD
:10ADD300D8B4F7DE58F6F8F6D6F6B5F676FE98F65A
:10ADE30097F697F6B6F6B5EEB5F6D7B4F1A4709428
:10ADF3000E5A885A47B553DE978BCD6AE9C5D4E618
:10AE0300F8D6557BCB4A246B49C613B5927BAA521D
:10AE130046CDD5DE97ACF0734983CB7B8A5AA752D4
:10AE2300875AE98C71ADB66BD07C538CF684B66BC4
:10AE3300F3530F42AE4ACE5B304ACE4A8E73B2848E
:10AE43001494B6A518A4F8ACD8B4F7DE38EED8EE4F
:10AE5300B6F6B5EE76F697F697F677F6B6F6B5EE5E
:10AE6300B5F6D7B512A490942F52267B8C9C6FCD48
:10AE7300F58BED5226AD51DED7CE357BAB62E79C29
:10AE8300AEB591E6F7A4EF5A8783ACCDF5E6B8B536
:10AE930031B531B5318C2D5AC85AEA8C51A5556359
:10AEA3008F8CF6849584B66BD25B715B504ACE521D
:10AEB300CE530F5B1073B27BD39496A4F89CD8B493
:10AEC300F8B517DE38EED7EEB5F6B5EE76F697F6AB
:10AED30097F677F6B6F6B5EE95F6D7B4F1A4908B60
:10AEE300CD8BED83CD8C0EC5B4AD118C0D840CB51B
:10AEF30051E6D7AD519CAE73AAA530DED6BDB3944F
:10AF03006F83CDA4D0C5D4E6D8CE15A4AFA4D08486
:10AF13000E73ADA5559D1574129D58745574344B1D
:10AF23000F533063B2533052EF6BB26B714A8E637F
:10AF3300318435A4F8A518B518BD17DE58EED8EE40
:10AF4300B6F6B5F676FE98FE98F697F6B6F6B5EE33
:10AF530095EEB7B4D19C4F7B4BBD5383CCACF1C5BD
:10AF6300D4C5D4B5527BABD656E6F7B592AD307B9C
:10AF7300CBDEB7CE349CCFA5116B2AAD32D636E6E5
:10AF8300B7DE97B57283ED83EE73ADAD7573F08461
:10AF93009484D67C9563D34AEF530F63924AAE32BF
:10AFA3000C635173D35AF0528E73929CB7A518B5A4
:10AFB30019BD17DE38EED8EEB6F6B5F676FE98F67E
:10AFC30097F697FEB6F6B5EEB5EEB6ACB09C2F7B12
:10AFD3004B9C8F946FBDB4BDB4A4F08C2E8C2DDE2E
:10AFE300D8AD51840C83EB9CAECE35B5B373AB8C2B
:10AFF3002D738BC5F4CE35C5F4CDF4B572944E9450
:10B003009094B1A555634E849474337C9663D36353
:10B01300926BD284966BB3426E637284557BF46BEE
:10B02300518435A518AD59B4F8BD17DE38EED7EE07
:10B03300B6F6B5F676F697F677F677F6B6F6B5EE94
:10B04300B5EED7B4D19C2F734B8C0D9C8FAD11CE25
:10B05300358C2D9C8F8C0DCE35D676948F9CCF9CC2
:10B06300D0BDD3D6979CD08C2D94AFBDD3BDB3CEDA
:10B0730014C5D3AD11B572B593C616A5556BAF7C88
:10B08300937C9484F784D67C756BD384767C556BE0
:10B09300927C1484356B9284148C769CD79CD7B4A1
:10B0A300F8B517DE38EED8F6D6F6D6F676F697F676
:10B0B30077F677F6B6F6B5EEB5F6D7B4F1A47083A6
:10B0C300AC8BED9C8F9C6FD656A4D0B572946EADAD
:10B0D30032DED8A4D0A4F08C4EBDD4CE769CF094AE
:10B0E300AF842CAD71DEB6D655DED6DED7BDB3AD9B
:10B0F30052B5B49D335B4D84B38D3685169DBA8DA1
:10B103001863B25B51531052F06BB373D36B72A5D8
:10B1130039AD59AD39AD39B4F8B517DE38EED8F6D7
:10B12300F7F6F7F696F6B7F6B8F697F6B6EE96EEA6
:10B13300B6F6D7BD12ACB09C6F6B09B5729C8FBDD0
:10B1430093BDB38C4EBDB39CAFB572C5F49CD0A474
:10B15300F0A4F0B572AD7294AFA53094AEAD30B536
:10B1630091CE34CE14CE35BDF5B5D5B5F7532C8D70
:10B17300158CF56C5385178CD774147C346BB35BC7
:10B18300316B927C148C769496949694979CB7BD6D
:10B1930038B4D6DE59E678DE56E675F6F8F6D7E625
:10B1A30076EEB7FF39EE97F6D8EEB7BD32A48F9C93
:10B1B3008F63099CD0948F6309A5118C2DAD318CBD
:10B1C3004E83ECBDD3944EA4F06B49840CA4F0835E
:10B1D300EC9CAE7369944DA4CFC5F4C635CE77CE3F
:10B1E30078B5F6BE386BAF741184D595378D179546
:10B1F30038951895188CB78C969D18A539B59AA5CE
:10B2030018A4F8B57AB559B4D6BD16EE9BBD346211
:10B21300A8940CE696EEB6F718EEB7ACD0ACB08BAC
:10B223008BD5D4BD11ACAFAD11736B4A4652667367
:10B233006BAD32C5D48C2D5246A510CE55A4F083E8
:10B24300EC4A25946ECE35ACF052457B8AA4CFBD33
:10B25300D3B573CE77B5D5C6378C91849273F095F9
:10B263001584B47C747C54741374137C3473F37337
:10B27300F3843473B26B517BB37B9294559CB6B415
:10B28300B5B4B4E65AD5F6940DB4F0E696E655EEA9
:10B2930096DE148B8BAC6F7B09DE15C5529C4EA4D6
:10B2A300B09CB0736B8C2EA4F1B552DE98B573B518
:10B2B30052A4D0AD31E6B8C5D4A4AFB552B531CEA2
:10B2C30035A4CF946E9C8FA4F0B5939CB09D127B54
:10B2D300EE73CE73EF52EC5B4E6BB08CB495167C71
:10B2E300548D179D38741373F39CF7A5189CB69C63
:10B2F300D79455A4D7AD39CD78C536CD97A4709CD6
:10B303002D9C0CC571EED6EE96E656A44EAC8F9BE3
:10B31300EDC552C552AC8FBD738C2E734BC5B4D6DD
:10B3230057D636A4D1AD12DE77B532BD93B5539C53
:10B333006FBD93BD73A4B09C6FA4D0D656AD1194CA
:10B343006E8C4E8C4F5AE95AEA3A0729A6320842C4
:10B353004A29C83A4A4AAD639074548CD68475849A
:10B363005494D6843473929CB68C35A4B7AD18AC80
:10B3730095BD36EE9BCDB6EEB8D614E696EED7E67F
:10B3830096F6F8CD93CD73CD93C552BD11BD11ACD7
:10B39300F183CD944FCDF6AD128BEE6AEAC5B4C5F9
:10B3A300D5B5338BCD62A9A4D1CDF69C7083CD7373
:10B3B3006BB553C5F5AD32736B4226420539C53AB9
:10B3C3000652A94A693A08298631C83A2A3209320B
:10B3D3002A196729C9530E845494B57BF37BD37B15
:10B3E300B27BB29C96A4F8BD17ACB5E67AE658E6F4
:10B3F30077ACCFACAF942CA48EBD119C0DC552EE8F
:10B40300B8EE97B4D0ACD0ACF2942F942FA4B19CE7
:10B4130070732B734CACF29C70A4B17B8D7BADB578
:10B42300339C90945083CD736CCE168C0E7BCD528F
:10B43300884A674A4794906B6C3A0729645AEB5AD7
:10B44300EC4A8B3A095B0D7432532E3A4B31EA5B6B
:10B453000E8C959CD69CD6A4D79CB6B539B539B578
:10B4630017ACD6D619E69ACDD59C4E942DACD09C6C
:10B473008E9C4E8BACACB1D616E6B8B512B4F1AD1A
:10B4830012A4D19CB19CB19C91945094709CB1A492
:10B49300F2AD13A4D294719471A4F3C5F78C509CAC
:10B4A300919CB19CD26B4C528842277BEE8C4F739C
:10B4B3008D6B4C6B6D845073AE7BEF4A6A52CC5BE1
:10B4C3006F5B8F4AED29C9426C8C749CF794B69CD0
:10B4D300D79455A4B7A4F8ACF8ACF77B90732D8B35
:10B4E300EE9CB0736B8C2D83ED8BED9C908BCE8398
:10B4F300AD7B6C62A962C96B0A62EA6B2B630A4A71
:10B5030027738C528962EB6B2B52A96B4C738D6B37
:10B513006D6B6D5AEB738D738D6B2C736D5AEA5291
:10B52300895289632B9D128C505AEA42275B0B6B1D
:10B533006E94B3528A424A5B4E3A8B320929E94AE6
:10B543008C6B706B70737162EF5AAF83F4AD189CA0
:10B55300B79CB76B4F62CC632B52A95AC96B2A6352
:10B563000A5A886B2B5A8952284A075A6852474A03
:10B57300274A4742274A684A884A684A684207393D
:10B58300E739E742485AEB5B0C4AAA4A6A52AA6374
:10B593000C526931A639E75ACA52AA52CA7BCE73F2
:10B5A300AD422842284A694A694A6A422952EC5BF9
:10B5B3004E4B0D4ACC428C424B3A0A420B422C5A18
:10B5C300CF526D7B92A4D8B57AAD397BB1630D634D
:10B5D3000C4A684226424752884206528942084A28
:10B5E3002852695ACA5AC94A474A684A6852A952EC
:10B5F300C952A94A89422842083A0842695AEC5B6F
:10B603000C52CB4AAB52CC6B6E62EC4A2939E84AF6
:10B61300494A4942284A895B0B4AAA4AAA3A28312D
:10B62300E8426A424A426A3A4B322A322A320A3A98
:10B633000A39EA39EA420B5AAF5A8E83D4B5399C98
:10B64300D894966B2F5AAC5ACB4A684A474A6752EA
:10B65300A94A2752894A4852695AAA5AA952685292
:10B66300A852885288528852A952A952894A694AD3
:10B673004942494A8A5AEC52EC52AB4AAB52CC5239
:10B68300AC528B4A4A39E842294A8A4A8A42494299
:10B69300694A8A4AAB3A0831E8426A426A426B3ADB
:10B6A3004B324B322B3A4B3A2C3A0B420B420C4A5D
:10B6B3002D4A2D7372A4B8AD39B559A4F6AD15B59D
:10B6C30095B594B573BDB4BDB4B553BD95B574B557
:10B6D30075B5549C918C0E9C908C2E8C0E83CD83CF
:10B6E300EE8C2F8C2F8C51843084318C518C728C46
:10B6F300528431843284528C528C538C327BF1735A
:10B70300D07C317C106BAE636D5B4D636E63AF6B4E
:10B71300AF638F63B07C537C747C747C547C54849F
:10B723005484148414841483D37BB39456AD19AC1A
:10B73300D7B558CE1ADE9AEEFAE6D9DE97DEB7DE33
:10B74300B7DE97E698E699E6B9E698BD53A4B1B596
:10B75300129C6F9C70940F942F9C719C51A4D39C4A
:10B76300B2A4B3A4B39CB49C9394939C949CB49CB4
:10B77300D59CD59CD59CD48C738C7384727C117CA2
:10B78300527C31743184D4953684B484D49D988C9E
:10B79300D684B68CB68CB694B794B79CD7A4F8A4C9
:10B7A300D79CB7A4B8A4F8B4F7BD37D63ADE9ADE6F
:10B7B30098DE97DE56E696DE76DE77DE57DE57E6D0
:10B7C30078E677BD32ACD1BD12A46FACB1A470A43E
:10B7D30091ACB29C50A4B3A4B3ACD4ACF4A4D4A4A1
:10B7E300B4A4B4ACF5AD16949494B49CD59CF59CD8
:10B7F300D58CB48C938CB37C32849374327C7384F5
:10B80300F57C947CB48D168D178CD78CD78CD794FC
:10B81300D79CD89CF8A519A4F9AD19AD19AD192079
:10B823000000000000000000000000000000000015
:10B83300220000000000001428285000000000002F
:10B84300002C000000000000181808300000000061
:10B8530000002D0000000000000000FE00000000BA
:10B863000000002E00000000000000181800000077
:10B8730000000000300000001824424242424242CD
:10B883002418000000310000001070101010101078
:10B8930010107C000000320000003C424202040809
:10B8A3001020427E000000330000003C4242041896
:10B8B300040242423C00000034000000080818283B
:10B8C30048487E08081E000000350000007E404006
:10B8D3005C62020242423C000000360000001C246D
:10B8E30040405C624242423C000000370000007E60
:10B8F3004444080810101010100000003800000025
:10B903003C4242423C244242423C00000039000097
:10B913000038444242463A020224380000003A000A
:10B923000000000018180000001818000000003B79
:10B9330000000000080000000000080810000000DC
:10B94300410000001010282828287C4444EE000001
:10B953000042000000FC4242447844424242FC0060
:10B963000000430000003E42828080808082443891
:10B9730000000044000000F8444242424242424474
:10B98300F800000045000000FC4248487848484061
:10B9930042FC00000046000000FC4248487848484A
:10B9A3004040E0000000470000003C448480808069
:10B9B3008E84443800000048000000EE4444447C78
:10B9C30044444444EE000000490000007C10101081
:10B9D30010101010107C0000004A00003E080808F8
:10B9E30008080808080888F000004B000000EE442F
:10B9F30048507050484844EE0000004C000000E0FE
:10BA03004040404040404042FE0000004D000000E6
:10BA1300EE6C6C6C5454545454D60000004E000029
:10BA230000EE64645454544C4C4CE40000004F004A
:10BA330000003844828282828282443800000050AF
:10BA4300000000FC4242427C40404040E0000000D5
:10BA53005100000038448282828282B24C38060050
:10BA63000052000000F84444447850484844E6003B
:10BA73000000530000003E424240300C0242427C30
:10BA830000000054000000FE92101010101010105F
:10BA93003800000055000000EE444444444444444C
:10BAA300443800000056000000EE4444442828288F
:10BAB30028101000000057000000D6545454546C52
:10BAC3002828282800000058000000EE44282810E9
:10BAD30010282844EE00000059000000EE444428DA
:10BAE3002810101010380000005A0000003E4404D3
:10BAF3000808101020227E0000005B00003C20207C
:10BB03002020202020202020203C00000040402036
:10BB130020101010080804040402005D00003C0417
:10BB2300040404040404040404043C005E00000050
:10BB3300000000001824000000000000005F000067
:10BB4300000000000000FE00000000000000600094
:10BB53000000000000003008000000000000006149
:10BB6300000000000038441C2444443E0000000050
:10BB730062000000C040405C62424242427C0000DE
:10BB8300006300000000001C22404040221C000013
:10BB93000000640000000C04047C848484848C769C
:10BBA3000000006500000000003C427E4040423C33
:10BBB30000000000660000000E12107C1010101030
:10BBC300107C00000067000000003E444438403C05
:10BBD30042423C00000068000000C040405C6242FA
:10BBE300424242E70000006900000030300070105C
:10BBF300101010107C0000006A00000C0C001C04E4
:10BC03000404040404447800006B000000C04040B6
:10BC13004E4850684844EE0000006C00000070106D
:10BC2300101010101010107C0000006D00000000B8
:10BC330000F85454545454D6000000006E00000021
:10BC43000000DC6242424242E7000000006F000055
:10BC53000000001824424242241800000000700033
:10BC6300000000DC62424242427C40E0000000717E
:10BC7300000000007C848484848C74040E00000023
:10BC8300720000000000EE3220202020F8000000A7
:10BC9300007300000000003C444038044478000076
:10BCA3000000740000000010107C10101010100C25
:10BCB300000000750000000000C642424242463BBD
:10BCC30000000000760000000000E7422424281052
:10BCD3001000000000770000000000D654545428E0
:10BCE3002828000000007800000000006E241818C7
:10BCF300182476000000007900000000E7422424A5
:10BD030028181010E00000007A00000000007E44B4
:10BD1300081010227E000000007B00001810101095
:10BD2300101020101010101018007C0010101010AC
:10BD330010101010101010101010107D0000301093
:10BD43001010101008101010101030007E000000AA
:10BD53000000000062928C00000000000000C9EEA9
:10BD6300400027FE2404012081185608504010404B
:10BD730027FC2040C0E04158464E584440404040D4
:10BD8300DBDA0000120412441244FE44124412444B
:10BD93001244124412443A44C444044408041004B0
:10BDA3000000CEB008400C40084017FC104033FCA4
:10BDB3003040504097FC1044104410441044105439
:10BDC30010481040C7B6010021083FF80000244086
:10BDD30024407E7C248425283C20242024503C4875
:10BDE300248E25040200BFC6060878880848084840
:10BDF300FE0818881C482A48280E48788B880808AB
:10BE03000808080808080808BCBC102010201020E7
:10BE1300FDFE1020142019FC3108D088109010600A
:10BE230010601090110E56042000B5E701000100C8
:10BE330001003FF8210821083FF8210821082108C3
:10BE43003FF821080102010200FE0000D7D30000E1
:10BE53003FF0002000400080010001000104FFFECC
:10BE63000100010001000100010005000200D3D020
:10BE7300010001007FFE020004000FF018102810DB
:10BE83004FF0881008100FF0081008900870082071
:10BE9300CFDE0000FBF8920893F8A208A20893F8FB
:10BEA3008A808A48AA50922082208210828E83043C
:10BEB3008200B9AB0000044006400440082008108B
:10BEC3001018220E430402000420081011F83F1832
:10BED30010100000CBBE00003FFC000400047FE410
:10BEE300000400043FC4204420443FC420442004F1
:10BEF300001400080000C9E4080810083F082108DE
:10BF03003FFE21083F08214821287F2805280908EA
:10BF13001108210845280210C6B5080008FE4E2066
:10BF2300484048FCFE8400A408A44AA44AA484A46C
:10BF3300085010482086C3020000BFA8010001007A
:10BF430001FC0100010001007FFE0100010001402E
:10BF530001300118010C010801000100BDC92108CD
:10BF6300320827C8445057DEF47417D4211447D439
:10BF7300F21403881A88E49404940AA61144B7D1EE
:10BF830002403FF802483FF822403FFE0442084A7D
:10BF93001FF4681009100910091002C00C38301082
:10BFA300CFB5007C3F800220042008401F8003207F
:10BFB3000C103FF8108C04A0089010882084428451
:10BFC3000100CDB31040102023FE20404440F888E8
:10BFD300090413FE20947C90009000901D12E1123E
:10BFE300020E0400D3E00100010002800460081087
:10BFF3003FFEC10401003FFC01001140193011183C
:10C00300211045000200B6EE100008FE7F9051207B
:10C013001EFE228254820C9212923E92E29222AA35
:10C0230022243E4221820000BAC51FF010101010D6
:10C0330010101FF00000FFFE080008001FF008109A
:10C0430000100010011000A00040D4AA00001FF847
:10C053000000000000007FFE044004400440044050
:0CC063000840084010422042403E00000F
:10DE9100420059020349004F0931000004110011E9
:10DEA1000045004805300000041A401A220004FF12
:10DEB100FFFFFFFFFF060000000000000000000060
:05DEC10001020304054D
:0BE08F00EF1FAC0670011E4C70F62263
:0BDFD9007C007E0012E05A7F327E00C8
:10DFE400AB07AA06EB1BAE0270011A4E60097F95BF
:08DFF4007E0012E08F80ED2297
:10E03B00AD07AC06C2A5C2A4ECF580C2A3D2A3ED7A
:09E04B00F580C2A3D2A3D2A522E4
:05E01D00E0FEA3E0FF9E
:10E02200AD07AC06C2A5D2A4ECF580C2A3D2A3ED83
:09E03200F580C2A3D2A3D2A522FD
:10DFFC0090000EE0FBA3E475F00112C6FCA9F0FA48
:04E00C0012C66CFFCD
:0DE01000C2A5D2A48F80C2A3D2A3D2A522A4
:07E09A00901C00E0FF7E0076
:01E0A100225C
:06E054007D077C007E0048
:0EE05A00AB05AA0412E03BAE02AF0302E022C7
:10D06300C2A1C2A67F0A7E0012DFE4D2A67D087C9D
:10D07300307FE37E0012E05A7D127C007FE77E0062
:10D0830012E05A7D317C127FEF7E0012E05A7D0060
:10D093007C017F017E0012E05A7D007C077F027EC7
:10D0A3000012E05A7D307C107F037E0012E05AE4C8
:10D0B300FDFC7F04FE12E05A7D077C027F087E00A0
:10D0C30012E05A7D007C077F097E0012E05AE4FDDE
:10D0D300FC7F0AFE12E05AE4FDFC7F0CFE12E05ACC
:10D0E300E4FDFC7F0DFE12E05AE4FDFC7F0FFE120F
:10D0F300E05A7DF07C007F107E0012E05A7F11120F
:10D10300E0547D967C007F127E0012E05AE4FDFC21
:10D113007F13FE12E05A7FC87E0012DFE47D907C0D
:10D12300147F107E0012E05A7D277C027F1112DFEC
:10D13300DB7D1D7F1212DFD97D007C1A7F137E00F9
:10D1430012E05A7D337C007F297E0012E05A7D0E67
:10D153007F2B12DFD9E4FDFC7F20FE12E05AE4FDB1
:10D16300FC7F21FE12E05A7F3012E0547D067C02E0
:10D173007F317E0012E05A7D067C057F327E0012ED
:10D18300E05A7D047C077F357E0012E05A7D037CE4
:10D19300127F367E0012E05A7D077C007F377E00C7
:10D1A30012E05AE4FDFC7F38FE12E05A7D067C074C
:10D1B3007F397E0012E05A7D017C077F3C7E00129E
:10D1C300E05A7D0F7C007F3D7E0012E05AE4FDFCB7
:10D1D3007F50FE12E05A7DEF7C007F517E0012E00B
:10D1E3005AE4FDFC7F52FE12E05A7D3F7C017F53DF
:10D1F3007E0012E05A7D007CA77F607E0012E05A19
:10D203007D017C007F617E0012E05AE4FDFC7F6AB1
:10D21300FE12E05A7D107C007F907E0012E05A7D62
:10D22300007C067F927E0012E05A7D037C007F9390
:10D233007E0012E05A7D107C017F957E0012E05A39
:10D24300E4FDFC7F97FE12E05AE4FDFC7F98FE129A
:10D25300E05A7D337C017F077E0012E05A7F647EB3
:10D263000012DFE4D2A190004D74FFF0A374E0F04C
:0AD2730090005B74F8F0A3E4F022D1
:05DEF4002DFDE03CFCE7
:10DEF9008D828C83AD07AC067F207E0012E05AAE7E
:10DF090083AF82AD07AC067F217E0012E05A7F22E3
:05DF19007E0002E03B68
:10DD2C00900028EEF0A3EFF0A3ECF0A3EDF0A3EA43
:10DD3C00F0A3EBF0900028E0FCA3E0FD7F507E0008
:10DD4C0012E05A90002CE0FCA3E0FD7F517E001203
:10DD5C00E05A90002AE0FCA3E0FD7F527E0012E026
:10DD6C005A90002EE0FCA3E0FD7F537E0012E05A97
:10DD7C00900028E0FEA3E0FFA3E0FCA3E0FD02DEA0
:01DD8C00F99D
:10DB800090000CE4F0A374E7F074FFA3F0A3F07D21
:0BDB9000C87BE67A007C007F787E00F6
:10DB9B00900006EEF0A3EFF0A3ECF0A3EDF0A3EAF8
:04DBAB00F0A3EBF008
:10DBAF00C007A3E0FFA3E090002ECFF0A3EFF0D0CB
:10DBBF000712DD2C900008E0FFA3E0900010CFF0DB
:10DBCF00A3EFF090000CE0FEA3E0FFD3900011E074
:10DBDF009F900010E09E5034900006E0FEA3E0FB03
:10DBEF00AA06C390000BE09B90000AE09A400D90AC
:10DBFF00000E12E01D0BBB00010A80E6900011E041
:0CDC0F0004F070BF900010E004F080B73B
:01DC1B0022E6
:10DF450090000C7401F0A37440F090005BE0FFA317
:10DF5500E090000ECFF0A3EFF07BF07A00E4FDFC3B
:05DF6500FFFE02DB9B42
:08DDEE00900003EEF0A3EFF03A
:10DDF60090002E7401F0A3743FF07BEF7A00E4FDEF
:10DE0600FCFFFE12DD2CE4FDFCFFFE12DEF9E490C1
:10DE16000005F0A3F0E4FBFA90000312E01D0BBB33
:10DE260000010ABA01F2BB40EF900006E004F07070
:10DE360006900005E004F0C3900006E094F0900020
:06DE460005E0940040CF4E
:01DE4C0022B3
:0ED80B00900012EEF0A3EFF0A3ECF0A3EDF00E
:10D81900E490001EF0A3F0A3F0A3F0A3F0A3F0A3FB
:10D82900F0A3744FF0E490001EF0A3F090001EE006
:10D83900FEA3E0FFC3944FEE9400502C12C66CFD7A
:10D8490090B82275F011EF12C75CEE75F011A4259E
:10D8590083F583E4936D601090001FE004F070CCB1
:10D8690090001EE004F080C4900024E0FEA3E0FFD5
:10D87900C390001FE09F90001EE09E400302D98FD5
:10D88900900012E0FAA3E0FBFFAE02C006C007A3B6
:10D89900E0FCA3E0FDEB2407FBE43AFA900014E076
:10D8A900FEA3E0240FFFE43E90002EF0A3EFF0D09A
:10D8B90007D00612DD2CE4900020F0A3F0900020A0
:10D8C900E0FEA3E0FFC39410EE9400400302D98F59
:10D8D90090001EE0FCA3E090B82375F01112C75C1C
:10D8E900EC75F011A42583F583E5822FF582E58394
:10D8F9003EF583E493F9E4900022F0A3F09000222E
:10D90900E0FEA3E0FFC39408EE9400506874807EA3
:10D9190000A807088006CEA2E713CE13D8F8FFE9BE
:10D92900FDEF5D6005900019800990001DE0700809
:10D9390090001B12E01D802C900022E0FEA3E0FF66
:10D94900900013E02FFF900012E03ECF2401CF3466
:10D9590000FE900020E0FCA3E0FD900015E090009F
:10D969001412DEF4900023E004F07091900022E09C
:10D9790004F002D906900021E004F070069000201E
:06D98900E004F002D8C624
:01D98F002275
:0ED27D00900012EEF0A3EFF0A3ECF0A3EDF0A2
:10D28B00E490001EF0A3F0A3F0A3F0A3F0A3F090A2
:10D29B000026F0A37417F0E490001EF0A3F09000AA
:10D2AB001EE0FEA3E0FFC39417EE9400505112C68C
:10D2BB006CFD90BD6175F022EF12C75CEE75F0222C
:10D2CB00A42583F583E493B5052590000112C6854B
:10D2DB00FF90001EE0FCA3E090BD6275F02212C728
:10D2EB005CEC75F022A42583F583E4936F601090BA
:10D2FB00001FE004F070A790001EE004F0809F90E8
:10D30B000026E0FEA3E0FFC390001FE09F90001EED
:10D31B00E09E400302D46D900012E0FAA3E0FBFF05
:10D32B00AE02C006C007A3E0FCA3E0FDEB240FFB9D
:10D33B00E43AFA900014E0FEA3E0240FFFE43E90E1
:10D34B00002EF0A3EFF0D007D00612DD2CE49000F6
:10D35B0020F0A3F0900020E0FCA3E0FD25E0FFEC23
:10D36B0033FE90001EE0FAA3E090BD6375F022122D
:10D37B00C75CEA75F022A42583F583E5822FF5823D
:10D38B00E5833EF583E493FAED25E0FFEC33FE9065
:10D39B00001EE0FCA3E090BD6475F02212C75CECAC
:10D3AB0075F022A42583F583E5822FF582E5833E74
:10D3BB00F583E493FFEAFE900024EEF0A3EFF0E494
:10D3CB00900022F0A3F0900022E0FEA3E0FFC394B4
:10D3DB0010EE9400506CE47E80A807088005CEC345
:10D3EB0013CE13D8F9FF900024E05EFEA3E05F4E4E
:10D3FB006005900019800990001DE0700890001BDB
:10D40B0012E01D802C900022E0FEA3E0FF900013A1
:10D41B00E02FFF900012E03ECF2401CF3400FE90AE
:10D42B000020E0FCA3E0FD900015E090001412DE5C
:10D43B00F4900023E004F07006900022E004F00268
:10D44B00D3D1900021E004F07006900020E004F0AE
:10D45B00C3900021E09410900020E0940050030250
:02D46B00D35F8D
:01D46D00229C
:04DAA7007DD0FCFE34
:10DAAB00900006EEF0A3EFF0A3ECF0A3EDF0A3EBE8
:10DABB00F0A3EAF0A3E9F090000AE0FBA3E0FAA3DD
:10DACB00E0F912C66CFF700302DB7FEFD3948090FA
:10DADB000008E0FCA3E0FD404890000DE0FFA3E050
:10DAEB00900019CFF0A3EFF090000FE0FFA3E090B0
:10DAFB00001BCFF0A3EFF0900011E090001DF09011
:10DB0B000006E0FEA3E0FF12D27D900007E0241098
:10DB1B00F0900006E03400F090000BE475F002800A
:10DB2B004DA3E0FBA3E0FAA3E0F9A3E0FFA3E09091
:10DB3B000019CFF0A3EFF090000FE0FFA3E09000EF
:10DB4B001BCFF0A3EFF0900011E090001DF09000C0
:10DB5B0006E0FEA3E0FF12D80B900007E02408F0CC
:10DB6B00900006E03400F090000BE475F00112C653
:05DB7B00E602DAC222FF
:10CCFF00900033EEF0A3EFF0A3ECF0A3EDF0A3EA76
:04CD0F00F0A3EBF0B2
:10CD1300FFAE02E4FCFD7B807A967998F812DE4D33
:10CD2300EF243090003FF0900037E0FEA3E0FFE4F3
:10CD3300FCFD7B807A967998F812DE4DAC00AD014C
:10CD4300AE02AF037B407A42790F780012DE4DEFDB
:10CD53002430900040F0900037E0FEA3E0FFE4FCB5
:10CD6300FD7B807A967998F812DE4DAC00AD01AE6A
:10CD730002AF037B407A42790F780012DE4DAC009C
:10CD8300AD01AE02AF037BA07A867901780012DE93
:10CD93004DEF2430900041F0900037E0FEA3E0FF18
:10CDA300E4FCFD7B807A967998F812DE4DAC00ADF9
:10CDB30001AE02AF037B407A42790F780012DE4D59
:10CDC300AC00AD01AE02AF037BA07A867901780097
:10CDD30012DE4DAC00AD01AE02AF03E47B107A2747
:10CDE300F9F812DE4DEF2430900042F0900037E066
:10CDF300FEA3E0FFE4FCFD7B807A967998F812DECF
:10CE03004DAC00AD01AE02AF037B407A42790F789F
:10CE13000012DE4DAC00AD01AE02AF037BA07A86FB
:10CE23007901780012DE4DAC00AD01AE02AF03E430
:10CE33007B107A27F9F812DE4DAC00AD01AE02AFDC
:10CE430003E47BE87A03F9F812DE4DEF2430900017
:10CE530043F0900037E0FEA3E0FFE4FCFD7B807A23
:10CE6300967998F812DE4DAC00AD01AE02AF037BAC
:10CE7300407A42790F780012DE4DAC00AD01AE026C
:10CE8300AF037BA07A867901780012DE4DAC00AD4A
:10CE930001AE02AF03E47B107A27F9F812DE4DAC42
:10CEA30000AD01AE02AF03E47BE87A03F9F812DECA
:10CEB3004DAC00AD01AE02AF03E47B64FAF9F812A6
:10CEC300DE4DEF2430900044F0900037E0FEA3E005
:10CED300FFE4FCFD7B807A967998F812DE4DAC0076
:10CEE300AD01AE02AF037B407A42790F780012DEC8
:10CEF3004DAC00AD01AE02AF037BA07A8679017819
:10CF03000012DE4DAC00AD01AE02AF03E47B107A3C
:10CF130027F9F812DE4DAC00AD01AE02AF03E47B9E
:10CF2300E87A03F9F812DE4DAC00AD01AE02AF03AF
:10CF3300E47B64FAF9F812DE4DAC00AD01AE02AF4A
:10CF430003E47B0AFAF9F812DE4DEF243090004532
:10CF5300F0900037E0FEA3E0FFE4FCFD7B807A96CF
:10CF63007998F812DE4DAC00AD01AE02AF037B4001
:10CF73007A42790F780012DE4DAC00AD01AE02AFFC
:10CF8300037BA07A867901780012DE4DAC00AD01F7
:10CF9300AE02AF03E47B107A27F9F812DE4DAC0042
:10CFA300AD01AE02AF03E47BE87A03F9F812DE4D7C
:10CFB300AC00AD01AE02AF03E47B64FAF9F812DE14
:10CFC3004DAC00AD01AE02AF03E47B0AFAF9F812EF
:10CFD300DE4DEB2430900046F0E4A3F090003EF0E9
:10CFE30090003EE0FFC394095075743F2FF582E42F
:10CFF3003400F583E024D0700890003EE0640870AC
:10D003005690003EE0FB75F004A4FF900034E02F3F
:10D01300FF900033E035F0FEC007900035E0FCA33D
:10D02300E0FD743F2BF9E43400FA7B01900039E012
:10D03300FFA3E090000DCFF0A3EFF090003BE0FFE3
:10D04300A3E090000FCFF0A3EFF090003DE090003D
:0FD0530011F0D00702DAAB90003EE004F08081CC
:01D0620022AB
:06DCA8007A007C007E0002
:10DCAE00900006EEF0A3EFF0A3ECF0A3EDF0A3EAE4
:04DCBE00F0A3EBF0F4
:10DCC200E4900011F0A3F090000CE0FEA3E0FFC38B
:10DCD200900012E09F900011E09E504D900006E0EF
:10DCE200FEA3E0FF900011E0FCA3E0FD900009E03C
:10DCF2002DFD900008E03CFC12DEF9E4FDFCD3901F
:10DD0200000BE09D90000AE09C400D12DFFC12DF48
:10DD1200FC0DBD00010C80E6900012E004F070A73B
:09DD2200900011E004F002DCC9DC
:01DD2B0022D5
:10D65A0090000374FFF0A37400F0A3748AF09000A2
:10D66A000CE4F0A37446F0900003E0F9A3E0FAA3F7
:10D67A00E090000EC9F0A3EAF0A3E9F07BF07A008B
:10D68A00E4FDFCFFFE12DCAE90000CE4F0A3745D36
:10D69A00F0A374F8F0A3E4F07BEFFA7D46FCFFFEFA
:10D6AA0012DB9B7BFF7A00790390000D74FFF0A3D5
:10D6BA0074E0F0A374F8F0A3E4F0A3F07D4AFC7FD1
:10D6CA0026FE12DAAB90000C7401F0A3743FF0A3AB
:10D6DA007407F0A374E0F07BEF7A007D5E7C00E4CF
:10D6EA00FFFE12DB9B90000374FFF0A37497F0A374
:10D6FA007452F090000CE4F0A37414F0900003E06C
:10D70A00F9A3E0FAA3E090000EC9F0A3EAF0A3E9B6
:10D71A00F07B787D6E7F7812DCA87BFF7A0079181F
:10D72A00E490000DF0A3F0A37407F0A374E0F0E412
:10D73A00A3F07D86FC7F8CFE12DAAB90000374FFA7
:10D74A00F0A37483F0A374CAF090000CE4F0A374FD
:10D75A0032F0900003E0F9A3E0FAA3E090000EC9CA
:10D76A00F0A3EAF0A3E9F07B327DB47F0F12DCA8C4
:10D77A0090000374FFF0A374AAF0A37412F090004F
:10D78A000CE4F0A3741EF0900003E0F9A3E0FAA3FE
:10D79A00E090000EC9F0A3EAF0A3E9F07B3C7A001E
:10D7AA007DEC7C007F0A7E0012DCAE12DB809000EA
:10D7BA000C7401F0A3740BF074FFA3F0A3F07DECDA
:10D7CA0012DB917BFF7A007921E490000DF0A3F03F
:10D7DA00A37407F0A374E0F0E4A3F07F5012DAA771
:10D7EA007BFF7A007926E490000DF0A3F0A374077A
:10D7FA00F0A374E0F0E4A3F07DF4FC7F50FE02DABB
:01D80A00AB72
:0CE07700EF4E6007EF1F70F81E80F522CE
:10DF6A0075CBFC75CA6975CDFC75CC69C2AD75C82F
:10DF7A0004EF1FAC0670011E4C600730CFFDC2CF04
:05DF8A0080EFC2CA2275
:10DEC70075CBDC75CA0075CDDC75CC00C2AD75C8E5
:10DED70004EF1FAC0670011E4C600F20CF08300AFC
:0DDEE700FAC2CAC2CF22C2CF80E7C2CA224F
:10DF8F00750808AD081508ED6016EE2EFEC297EF66
:10DF9F00339295EF2FFFA296E4334EFED29780E394
:04DFAF00D297AF0650
:01DFB300224B
:0EE06800C2937FAA12DF8F7FFF12DF8FD29349
:01E076002287
:0DD990007F647E0012DF6A7B007A0079223E
:0BD99D00900003EBF0A3EAF0A3E9F018
:10D9A800E4900007F0900006F0900006E0FCC394B5
:10D9B80064501912E068EFB4F00374FDF07F0A7E3A
:10D9C8000012E077900006E004F080DDEC64FE6071
:10D9D8000302DAA4C2937FBB12DF8F900006EFF038
:10D9E800900003E0FBA3E0FAA3E0F9740112C6B2C9
:10D9F800E4900006F0900003E0FBA3E0FAA3E0F94E
:10DA080012C66CFF900006E0C39F50457FFF12DFEF
:10DA18008F900003E0FBA3E0FAA3E0F9A3E0FEF592
:10DA280082758300EF12C6C4900007E0FF8E8275EE
:10DA3800830012C685FEEF6E900007F012C66CD305
:10DA480094204005D2937F0122900006E004F080E4
:10DA5800A47F0A7E0012DF6A7FFF12DF8F90000327
:10DA6800E0FBA3E0FAA3E0F9A3E0F582758300EFF9
:10DA780012C6C47F0A7E0012DF6AD293900003E0C8
:10DA8800FBA3E0FAA3E0F9A3E0F58275830012C6D0
:0EDA980085FF900007E0B507037F00227F01A5
:01DAA600225D
:10DD8D007B007A007940900000EBF0A3EAF0A3E964
:01DD9D00F095
:0BDD9E00900003EBF0A3EAF0A3E9F013
:10DDA900E4A3F0C2937FCC12DF8FE4FC900003E080
:10DDB900FBA3E0FAA3E0F912C66CFEECC39E501A6D
:10DDC900900006E0FE8C8275830012C685FFEE6F17
:10DDD900900006F012DF8F0C80D2900006E0FF124F
:04DDE900DF8FD29363
:01DDED002213
:0CE08300C2927F327E0012DEC7D29222D1
:10D46E00E4789DF608F60812C7434352800012DF97
:10D47E00B412E0837FF47E0112DF6A12D063E4FF00
:10D48E00FE12DDEE12D65A2094FD784A7C007D0005
:10D49E007B007A00799F7E007F0412C646900000C2
:10D4AE00E4F0A37400F0A37440F07B007A00F9124C
:10D4BE00DD9E12D990789CA607900000E0FBA3E0B9
:10D4CE00FAA3E0F990000112C685FF7823E6B507AE
:10D4DE0005789CE6601312DD8D12D990789CA60714
:10D4EE007F647E0012DF6A80D0789EE66401184663
:10D4FE00700302D6592094FD7F467E0012DF6A200B
:10D50E0094E790000074FFF0A37400F0A37440F051
:10D51E007BFF7A00F912DD9E12D990789CA6077FC8
:10D52E002C7E0112DF6A789F7C007D007B007A00E2
:10D53E0079247E007F0412C646789F12C712E4FB40
:10D54E00FA79C078BF12C076789F12C72BE4FFFE1F
:10D55E00FDFC789F12C71E12C167501E7F007E8091
:10D56E007D527C43789F12C71E12C167600C400A21
:10D57E00789D760008760102D4F7784A7C007D000B
:10D58E007B007A00799F7E007F0412C64612DD8DE5
:10D59E0012D990789CA6077FC87E0012DF6A900091
:10D5AE000674FFF0A37400F0A3742BF0789F12C7DB
:10D5BE001290000912C7377B007A00797C12C8E1FD
:10D5CE007BFF7A00798812DD9E7BFF7A007931E449
:10D5DE0090000DF0A3F074FFA3F0A3F0E4A3F07F8E
:10D5EE007D12DAA77B007A00797CE490000DF0A31F
:10D5FE00F074FFA3F0A3F0E4A3F07DF4FC7F7DFEB6
:10D60E0012DAAB7BFF7A00793AE490000DF0A3F0CA
:10D61E0074FFA3F0A3F0E4A3F07DF4FC7FB4FE123C
:10D62E00DAAB7FD07E0712DF6A12DB8090000C74BB
:10D63E0001F0A3740BF074FFA3F0A3F07BE67A0065
:0BD64E007DEC12DB9512DB8002D50D95
:01D6590022AE
:10DFB400C2AD75C804758780759870758921758D93
:10DFC400FD858D8BD28EC2ABD2AFC2A8D288C2CA15
:05DFD400D2ACC20A22DC
:10C06F0002C209E86480F8E933E83360110460F034
:10C07F00ED33EC337009E8FCE9FDEAFEEBFF220437
:10C08F0060DED3EB9FEA9EE99DE8C2E78CF0C2F732
:10C09F0095F0400CE8CCF8E9CDF9EACEFAEBCFFBFE
:10C0AF0012C1D485D0F05804700320D5B3E80470C2
:10C0BF00075002B2D502C21392D5EC0460F7E4CC5C
:10C0CF00C0E0C398F8603B94186008400DD0E0FBC7
:10C0DF0002C1EBE4FBFAC9FC8028E830E406E4C9AE
:10C0EF00FBE4CAFCE830E305E4C9CACBFCE854071B
:10C0FF006010F8C3E913F9EA13FAEB13FBEC13FC26
:10C10F00D8F130F52FC3E49CFCEF9BFFEE9AFEEDC8
:10C11F0099FDD0E0FBEF4E4D4C701222DB0302C2B3
:10C12F0010EC2CFCEF33FFEE33FEED33FDED30E77B
:10C13F00EB02C1EBEF2BFFEE3AFEED39FDD0E0FB4A
:10C14F0050130BBB000302C213ED13FDEE13FEEFF2
:08C15F0013FFEC13FC02C1EB1D
:10C1670074F8CC6480CCC86480C8F582046043C38B
:10C17700EB9FF5F0EA9E42F0E99D42F0E89C45F01E
:10C1870060305018E5825FFFE582F42B5582FB5043
:10C19700210ABA001D09B90019088016E5825BFB60
:10C1A700E582F42F5582FF50090EBE00050DBD0034
:10C1B700010CC3EB9FF5F0EA9E42F0E99D42F0E8DF
:0DC1C7009C45F06007CC4820E701B3EC2256
:10C87C00E5082406F582E43400F583E005082290EF
:10C88C000003300703900006E475F00112C768023C
:10C89C00C66C2000E97F2ED2008018EF540F249034
:10C8AC00D43440D4FF30040BEF24BFB41A0050032F
:10C8BC002461FFE50960021509050CE50C70020501
:10C8CC000B30070E900003E475F00112C768EF02FD
:10C8DC00C6B202DF1E7403D2078003E4C207F50858
:10C8EC0090000312C77FE4F509F50BF50CE5096020
:10C8FC00077F2012C8BF80F5750AFFC201C200C2B3
:10C90C0002C203C205C206C20812C88BFF700D30EA
:10C91C0007057F0012C8D0AF0CAE0B22B4255FC246
:10C92C00D5C20412C88BFF24D0B40A00501A75F07B
:10C93C000A780930D50508B6FF0106C6A426F620EC
:10C94C00D5047002D20380D924CFB41A00EF50045E
:10C95C00C2E5D20402CBC2D20180C6D20080C0D2C2
:10C96C000280BCD2D580BAD20580B47F2012C8BF59
:10C97C002002077401B5090040F112C87CFF12C8EF
:10C98C00BF02C8F9D208D206809512C87CFB12C827
:10C99C007CFA12C87CF94A4B700679C07ACC7BFFC2
:10C9AC0020022EE509602A7E008E8275830012C655
:10C9BC008560060EEE650A70F0C2D5EBC0E0EAC0E9
:10C9CC00E0E9C0E0EE12CC23D0E0F9D0E0FAD0E000
:10C9DC00FB12C66CFF60AAEBC0E0EAC0E0E9C0E065
:10C9EC0012C8BFD0E02401F9D0E03400FAD0E0FB4B
:10C9FC00E50A0460DCD50AD98087D20280A212CC69
:10CA0C000560F7E50A70010412C21EA90A600DE563
:10CA1C000A600914F50A12CCADEF60F3EA30E702B4
:10CA2C00F404C3995079EAF4250A0430E701E404CC
:10CA3C00F50A800D12CC0560C1EA050A250A12C25E
:10CA4C001EEA900032F030E701E4250A04D50A040E
:10CA5C002005011412CC23E4C0E012CCAD900032BE
:10CA6C00E0601320E70714F012C8A7802204F0D06E
:10CA7C00E014C0E07F0012C8A7E50A600712C89E48
:10CA8C00150A800B30050312C89ED0E002C8F9D0FD
:10CA9C00E00480C412CC05609EE50A0412C21E900C
:10CAAC000032EAF0E50A200502600104240412CCED
:01CABC002356
:10CABD0074FF04C0E012CCAD12C8A7E50A20050230
:10CACD00600312C89ED0E0B50AE87F4512C8B19048
:10CADD000032E07F2B30E7047F2DF404C0E012C854
:10CAED00BFD0E075F00A84C0F012C8A8D0E012C81B
:10CAFD00A802C8F9791080027908C206C208800818
:10CB0D00D2D5790A8004790AC2D5E50A047002F5F6
:10CB1D000AE4FAFDFEFF12C87CFC7B08200113120B
:10CB2D00C87CFD7B1030000A12C87CFE12C87CFF49
:10CB3D007B20EC3382D592D55013C3E43000069F91
:10CB4D00FFE49EFEE42001039DFDE49CFCE4CBF894
:10CB5D00C201EC700CCFCECDCCE824F8F870F38088
:10CB6D0017C3EF33FFEE33FEED33FDEC33FCEB3348
:10CB7D00FB994002FB0FD8E9EB300105F8D0E0C47A
:10CB8D0048B201C0E00AEC4D4E4F78207B0070C2D8
:10CB9D00EAB50A0040BCC0E012CC25D0F0D0E020B0
:10CBAD000104C4C0E0C4B201C0F012C8A8D0F0D5D1
:10CBBD00F0EB02C8F912C788C99653CB0158C96763
:10CBCD004CC96342CB054FCB0D44CB0D49C97C43BA
:10CBDD00CB1355CA4046CAA045CA0A47CCE050C936
:10CBED006B2DC96F2EC9922BC97323C99020CCC947
:10CBFD002AC92B480000C98AE50AB4FF03750A0645
:10CC0D0012C87CFC12C87CFD12C87CFE12C87CFFC9
:10CC1D0090002B02C25B790AA2D5200314300509BE
:10CC2D00B910020404B9080104A2D520060250016E
:10CC3D00042002689202B509005034C0E07F203014
:10CC4D0003197F30A20272067205500F12CC7CC2FE
:10CC5D0002C206C205C2087F30800F300503E9C04D
:10CC6D00E012C8BF300503D0E0F9D0E0B509CC30F3
:10CC7D0005177F30B9100C12C8BF7F583004077FDD
:10CC8D00788003B9080312C8BF3002057F2D02C892
:10CC9D00BF7F202008F87F2B2006F322920280CF41
:10CCAD007F00B40700500B242BF582E43400F5838C
:10CCBD00E0FF22286E756C6C2900D20112C87C3001
:10CCCD0001F8C201780930D50108F602C92B2D50A3
:10CCDD0043495812C87C2403B405004001E490CCAC
:10CCED00DB9312C8B0743A12C8B0D20375090402AE
:02CCFD00CB0169
:10C1D400E9D2E7C933E833F892D5EDD2E7CD33ECB1
:07C1E40033FC5002B2D5222A
:10C1EB00EC30E7100FBF000C0EBE00080DBD0004B5
:10C1FB000BEB6014A2D5EB13FCED92E7FD2274FF61
:10C20B00FCFDFEFF22E480F8A2D574FF13FC7D80B9
:03C21B00E480EFCD
:10C21E00F920E73624F950037907E4F42402FBE50C
:10C22E0082158270021583DBF6E024FB501BE96059
:10C23E0014E4F0E582158270021583E004F0B40A6E
:0DC24E0008E4F0D9EE7401F00A22C2D522F6
:10C25B00ED33EC3392D5FA602AB4FF33EDC2E77BB2
:10C26B00FF60067AC27980E4227AC2798920D504EC
:10C27B007AC27984224E614E002B494E46002D49DD
:10C28B004E4600E47A08F0A3DAFC7B00740722C068
:10C29B0083C082ECC0E0EDC0E0EEC0E0EFC0E0EAAE
:10C2AB0075F010A4CAABF075F04DA42BFBE435F080
:10C2BB00FCEA2410FAEB34C5FBEC34D9FCEDC2E7F5
:10C2CB00FF75F056A4F42411C5F0F434C58FF0A417
:10C2DB002AE5F03BE43CF020E71412C536D0E0FF32
:10C2EB00D0E0FED0E0FDD0E0FC12C4698014F40471
:10C2FB0012C536D0E0FFD0E0FED0E0FDD0E0FC125E
:10C30B00C360D082D083E0FAEDD2E7CD33EC332497
:10C31B0082FBE4C3CF33CFCE33CECD33CD33DBF380
:10C32B007B0775F00A846004F0A31B0AE5F0F0A309
:10C33B008FF0740AA4FFACF08EF0740AA42CFEAC40
:10C34B00F050010C8DF0740AA42CFDE435F0F0A331
:05C35B00DBDE74072287
:10C36000EC4D6011E8497017ED33EC3304600DE4D7
:10C37000FCFFFEFD22E933E8330470F802C2091223
:10C38000C1D458046009E4CC248150062850090225
:10C39000C21328400302C210C0E0EB4A7044B980C7
:10C3A00006D0E0FB02C1FFEF4E701CBD8008EBFF22
:10C3B000EAFEE9FD80EBE98DF0A4FEE5F002C44958
:10C3C000E9CDF9EAFEEBFFEF89F0A4FCE5F0CE89B8
:10C3D000F0A42EFFE435F0CD89F0A42DFEE435F075
:10C3E0008067EF4E7005BD80D780C3EF8BF0A4ACA3
:10C3F000F0EE8BF0A42CFCE435F0F8EF8AF0A42CDE
:10C40000E5F038FCE433CB8DF0A42CFCE5F03BF8F0
:10C41000EE8AF0A42CFCE5F038F8E433CF89F0A4E0
:10C420002CFCE5F038CF3400CE89F0A42FFFE5F0E6
:10C430003EFEE433C98DF0A42EFEE5F039CD8AF03E
:10C44000A42FFFE5F03EFEE43DFD33D0E0FB5007B6
:10C450000BBB000F02C213EC2CFCEF33FFEE33FEDC
:06C46000ED33FD02C1EB0B
:10C4660002C213EC5D046005E85904700302C209B8
:10C4760012C1D4580460F6EC4860F2EC7004FDFE7C
:10C48600FF22C860DB2481C85009C39860025006A9
:10C4960002C2109850CAF582E9294B4A7005AB8250
:10C4A60002C1FF75F0007C1A7880C3EF9BEE9AED0F
:10C4B60099400DC3EF9BFFEE9AFEED99FDE842F021
:10C4C600DC23ACF0D0E0FFD0E0FED0E0FDAB822074
:10C4D600E7101BEB60BAEC2CFCEF33FFEE33FEEDFE
:10C4E60033FD02C1EBE803F830E705C0F075F00054
:10C4F600EF2FFFEE33FEED33FD40B830E7C280AAE2
:10C506003F8000004120000042C80000447A00003D
:10C51600461C400047C35000497424004B189680BF
:10C526004CBEBC205A0E1BCA6753C21C749DC5AEB6
:10C53600FB60065407601C232312C564EB54386065
:10C546000912C55012C55F12C360ECF8EDF9EEFA98
:10C55600EFCB22EB12C55F80F1543803241C90C543
:10C5660006FE93FC0EEE93FD0EEE930ECE93FF2287
:0300000002DC1C03
:0CDC1C00787FE4F6D8FD7581A202DC637D
:10C57600E709F608DFFA8046E709F208DFFA803EA7
:10C5860088828C83E709F0A3DFFA8032E309F60894
:10C59600DFFA8078E309F208DFFA807088828C83FC
:10C5A600E309F0A3DFFA806489828A83E0A3F608B0
:10C5B600DFFA805889828A83E0A3F208DFFA804C8A
:10C5C60080D280FA80C680D4806980F28033801061
:10C5D60080A680EA809A80A880DA80E280CA8033CA
:10C5E60089828A83ECFAE493A3C8C582C8CCC58342
:10C5F600CCF0A3C8C582C8CCC583CCDFE9DEE78012
:10C606000D89828A83E493A3F608DFF9ECFAA9F090
:10C61600EDFB2289828A83ECFAE0A3C8C582C8CCE6
:10C62600C583CCF0A3C8C582C8CCC583CCDFEADEFF
:10C63600E880DB89828A83E493A3F208DFF980CC61
:10C6460088F0EF60010E4E60C388F0ED2402B4045A
:10C656000050B9F582EB2402B4040050AF23234501
:06C66600822390C5C6739B
:10C66C00BB010689828A83E0225002E722BBFE02CC
:09C67C00E32289828A83E49322FF
:10C68500BB010CE58229F582E5833AF583E022506A
:10C6950006E92582F8E622BBFE06E92582F8E222B4
:0DC6A500E58229F582E5833AF583E49322CE
:10C6B200BB010689828A83F0225002F722BBFE0167
:02C6C200F32261
:10C6C400F8BB010DE58229F582E5833AF583E8F0AC
:10C6D400225006E92582C8F622BBFE05E92582C858
:02C6E400F22240
:10C6E600C5F0F8A3E028F0C5F0F8E58215827002DF
:06C6F6001583E038F0227C
:10C6FC00A3F8E0C5F025F0F0E582158270021583F1
:06C70C00E0C838F0E8224D
:10DE4D00C2D5E830E70FB2D5E4C39BFBE49AFAE400
:10DE5D0099F9E498F8EC30E717B2D512DE8312C7C2
:10DE6D00EAE4C39BFBE49AFAE499F9E498F8800399
:10DE7D0012C7EA30D50DE4C39FFFE49EFEE49DFD7D
:04DE8D00E49CFC22F3
:0CC71200E6FC08E6FD08E6FE08E6FF2253
:0DC71E00E6FB08E6F908E6FA08E6CBF8228B
:0CC72B00ECF608EDF608EEF608EFF6223A
:0CC73700ECF0A3EDF0A3EEF0A3EFF02275
:10C74300D083D082E493F608740193F608740293BD
:09C75300F608740393F6740473F4
:0CC75C00A42582F582E5F03583F58322E8
:10C76800F8E0FBA3A3E0F925F0F0E582158270025A
:07C778001583E0FA38F022FE
:09C77F00EBF0A3EAF0A3E9F022BB
:10C78800D083D082F8E4937012740193700DA3A340
:10C7980093F8740193F5828883E473740293686054
:06C7A800EFA3A3A380DF54
:10DF1E00EFB40A07740D12DF29740A309811A8990C
:10DF2E00B8130CC2983098FDA899C298B811F63063
:07DF3E0099FDC299F599223B
:10DC280002D46EE493A3F8E493A34003F68001F2D0
:10DC380008DFF48029E493A3F85407240CC8C333FD
:10DC4800C4540F4420C8834004F456800146F6DFCC
:10DC5800E4800B010204081020408090DE91E47EED
:10DC6800019360BCA3FF543F30E509541FFEE493C1
:10DC7800A360010ECF54C025E060A840B8E493A388
:10DC8800FAE493A3F8E493A3C8C582C8CAC583CAB3
:10DC9800F0A3C8C582C8CAC583CADFE9DEE780BE6B
:01DEC600005B
:10C7AE0075F008758200EF2FFFEE33FECD33CDCC42
:10C7BE0033CCC58233C5829BED9AEC99E5829840C5
:10C7CE000CF582EE9BFEED9AFDEC99FC0FD5F0D6A2
:10C7DE00E4CEFBE4CDFAE4CCF9A88222B800C1B9CC
:10C7EE000059BA002DEC8BF084CFCECDFCE5F0CB0A
:10C7FE00F97818EF2FFFEE33FEED33FDEC33FCEB43
:10C80E0033FB10D703994004EB99FB0FD8E5E4F9FD
:10C81E00FA227818EF2FFFEE33FEED33FDEC33FCEA
:10C82E00C933C910D7059BE99A4007EC9BFCE99ADE
:10C83E00F90FD8E0E4C9FAE4CCFB2275F010EF2F23
:10C84E00FFEE33FEED33FDCC33CCC833C810D70723
:10C85E009BEC9AE899400AED9BFDEC9AFCE899F85E
:0EC86E000FD5F0DAE4CDFBE4CCFAE4C8F922F1
:00000001FF
